:020000041100E9
:10300000002370B5284C0120636101F02DFA4020A7
:103010000223FE21254A207401F0ACFA002833D1A6
:103020000223FF21224A207C01F0A4FA00282BD1A0
:10303000204BA2899A4224D1E3891F4A93420CD1A2
:103040001E4B63611E4B2268002A03D1002B01D066
:1030500023CB23C401F07CFA70BD1A4A934201D0FD
:103060000023F0E7184B194A1B68934205D9C02288
:103070000421207C920001F0F7FA104B6361144B9D
:10308000E1E700232374EBE7CC223820AC21920146
:10309000207401F0E9FA0028F3D10E4B63610E4B66
:1030A000E3810E4BCFE7C0468863FF1F9463FF1F89
:1030B0009663FF1F5959000083050000C9420011A3
:1030C00094BE001182150000AC63FF1F871300003F
:1030D000A0BE001165430011AAAAFFFF88BE00111F
:1030E000F7B5164B0192C318021D002000938823E8
:1030F0005B05D3181B685C1C1AD09CB2402C18D8F6
:103100008D781E0CAC466746CD782D023D43AE420D
:1031100006D1019800280ED110000C70240A4C70C2
:1031200003249BB20733A343D218009B9A42DED3F9
:10313000FEBD4432F9E71000FAE7C046FC0F00007C
:10314000802213B503000324019189B25201073193
:103150009B18A14304305A1A88235B05C3181B68C7
:10316000591C03D190429241104016BD99B240299A
:1031700007D80B000733A343C0189042ECD30020BC
:10318000F3E74430F9E7134B134A1B68126810B594
:10319000FA24934201D81A00F824104BE4021B6869
:1031A0009A4210D813000E4A12689A420ED3013385
:1031B00007D1F823DB029C4203D10A49054808F0F5
:1031C00067FC200010BDFC24E402ECE7FE24E402CE
:1031D000F7E7C04600C0071100D0071100E0071153
:1031E00000F00711FFFFFF7FF0B59BB015000490C2
:1031F0000391402A00D9A0E006AB59801A80FFF75E
:10320000C2FF0400042816D9002206A9FFF768FFB0
:10321000052810D906AB1B88AB420CD1002D07D076
:10322000514B2A000499C01808F08AFA002802D1EC
:1032300001201BB0F0BD06AB1D8020000699FFF7F2
:103240007FFF041E7BD1069B0793FFF79CFF802323
:103250005B01C618802307001B039E4201D3F8269A
:10326000F60288235B05F31801931B68013302D033
:10327000019808F05DFB3D49019808F009FC3B1DF1
:103280000293331D05938822029B52059B181B68ED
:1032900008935A1C3CD044219AB20091402A04D889
:1032A0000320D11D814389B2009103991B0C8B42ED
:1032B00024D0402A22D80122300008A9FFF710FFAD
:1032C000021E1BD1380008A9FFF70AFF04000428DA
:1032D00031D9009A059B9B1880225201B218934263
:1032E00040D288235B05C118009A09A808F080FA2B
:1032F0001D4B009A09A9F01808F042FB009A029BA6
:103300009446634402931A4B029AFB189A42BAD32A
:1033100088235B05FC1821680198013908F0B8FB87
:10332000200008F005FB039A07AB5A80300007998C
:10333000FFF706FF0400002C03D1002079E70428E2
:10334000FBD988235B05E018069908F0A1FB03234D
:10335000EA1C9A4300D16BE7034B0499E01808F08C
:103360000FFB65E70424ECE704000011FFFFFF7F7B
:10337000F80F0000F7B505001400402A21D80027F7
:1033800001AE71803780FFF7FEFE042816D93A009F
:103390003100FFF7A5FE042810D93688BC420BD0B7
:1033A000BD4209D0221CB44200D9321C064B92B255
:1033B000C118280008F01CFA30B2FEBDC04300B2AC
:1033C000FBE703204042F8E70400001137B5042270
:1033D00004000D0001A81649FFF7CCFF02000428E5
:1033E0000BD1019BA34208D3AB4204D0104901A8E2
:1033F0000195FFF7F9FE01203EBD0E4C2368200029
:10340000019308F095FA019920000139019108F023
:103410003FFB80235B01E418074B9C42EED1042262
:10342000034901A80195FFF7DFFE0020E4E7C0464D
:103430005555000000C007110000081130B589B0D3
:1034400008F0AEFC10226946254808F009FC254B1F
:10345000009A9A420ED1019B029A0F2B33D8002179
:1034600001240698013B08D2002900D00292029B59
:10347000013331D10023029325E0551CF2D1020023
:103480002100EFE710341022200004A908F0E8FB27
:10349000029B013301D1069B0293882304995B05AB
:1034A000C918059B06981A03120B049105928142D4
:1034B00003D02B4201D108F09BF9019B013B019302
:1034C000019B002BDED1029B002B03D004930498B8
:1034D0004168084709B030BDE025014C2D03EFE7F6
:1034E0000000011150485936F7B50F490F4B0A68D3
:1034F00004001A4084235B0013430B60030003277E
:103500001033019300252E00112008F001FC084B18
:103510001B683B40AB4002351E43202DF4D1019B7C
:1035200040C4A342EED1F7BD5CF0004000FEFEFFB8
:1035300064F00040802270B5AD4CAE4BD20000214B
:1035400020001C6008F0FCFB2300AB4A88331A60A3
:10355000AA4B1A786E23002A00D01133E3620A23A3
:103560002365A74B1878A74BA0630138E361C3B26A
:10357000032B01D810232362A34B37226361C82396
:10358000DB00A36123008C331A60082336210F3A35
:10359000E518E16323646264E9670439251DE9677E
:1035A00025003B26BC352E602500C0352B6025004C
:1035B000C4352A6025000636CC352E602500083E2D
:1035C000C8352E602500D03529602100D4310B602C
:1035D0002100D8310A6021000225E0310D6025006C
:1035E0004221DC35296025001B3EE4352E60250094
:1035F000E8352B602500EC352A6022000525F432E1
:1036000015602200F03211602200183190321160F2
:1036100022009432136023003C2298331A60AF23B7
:10362000DB002360794B2363032805D808F058FAA0
:10363000330235371523636096232100FA225B009D
:10364000A360E360C8332361714BFC319200A36433
:103650000A6062626F4A704DA2627322E2656D3A3F
:103660006265A2650232E5644A60022161669621C4
:103670008900A166626709210022E166A2676749A5
:10368000674A684E2167E2673560032811D808F061
:1036900027FA96089EA61023CDE70E23CBE70C232E
:1036A000C9E720001A259C30056020000735A030AE
:1036B00005602000A83003602300FA20F833800062
:1036C000186023006420A433186023005F38AC33F3
:1036D000186023000338B03318602300C630B433B9
:1036E000186023000020B833186023003825FC330D
:1036F0009D604D4D5A665D644C4D9A64DD61962522
:10370000AD001D624A4D9A675D62F53DFF3D9D62C9
:103710001E25484ADD6618675867D9651966DA6755
:10372000BE23C021444A5B00E250444B4900635031
:1037300004316250C4225200A350FA23E4205B00FB
:103740000432A3500432A3503D493E4A3E4BD1605F
:103750003E49800019503E49E938FF3819503D492B
:10376000043019503C491038D1613C4911633C493F
:1037700051633C4911603C49195019003B48F831EC
:1037800008603B49D16582213A4A89005A501A00A3
:1037900039490832D1671A003849B432116088219A
:1037A000374A89005A501A00364988321160364A21
:1037B000DA6408F0D5F8012008F012FA70BD200094
:1037C00014259C30056020000435A03070E72000EF
:1037D00010259C30056020000335A03068E72000EC
:1037E0000E259C30056020000235A03060E7C04601
:1037F0000004FF1F6466FF1F5071FF1F1C46FF1F60
:103800004A0AFF1F3A07000080C3C9019A0200005C
:1038100050C300006A180000280A0000204E000073
:1038200088130000F009FF1F00400011681000001D
:10383000C4090000DC05000040420F001027000012
:10384000FD1BFF1FFC00FF1F0000FF1F252FFF1F98
:103850004D32FF1FE530FF1FD91FFF1FF51FFF1F50
:10386000A121FF1F491FFF1FC528FF1F8D2CFF1F10
:10387000D918FF1FD127FF1F3925FF1F4525FF1F1F
:10388000491EFF1F011FFF1FC11DFF1FF7B50B0CB6
:10389000FF270122009300233C001E001D009446D8
:1038A000019089B262469A401000084018413618CB
:1038B000B6B2FF2F02D1012E00D19FB20098024074
:1038C0001A41AD18ADB2FF2C02D1012D00D19CB22E
:1038D0000133102BE6D10320012E07D1012D04D195
:1038E000019B2401E4191C700138FEBD102EFCD18F
:1038F0000238102DF9D00230F7E710B5064C2378C6
:10390000002B07D10548FFF7EFFD0548FFF7ECFD59
:103910000123237010BDC0462466FF1F3866FF1FB9
:103920002866FF1FF0B58BB00D0001230190102910
:1039300036D8FFF7E2FF00231A001B48C15C0133B1
:103940005218102BFAD1023B002A29D0174B184CE1
:103950001F68002306A9E25C1600FA5C56405E541C
:103960000133102BF7D102AA08F09AF82A0002A915
:10397000019808F00DFA08F03BF823681B18236043
:1039800008F036F863681B18636008F031F8A36824
:103990001B18A36008F02CF8E3681B18E3600023F1
:1039A00018000BB0F0BDC0463866FF1FBC44FF1FB7
:1039B0002866FF1F0223F0B501245D4D5D4E2B707C
:1039C0005D4B91B01C705D4F039333680820BB7052
:1039D00006F052FC0023984205D0BA78552A02D04E
:1039E000332A00D098E03360002006F0DDFE07F0B7
:1039F000D7FEFFF79FFD07F003FF1F2201240021E0
:103A00004F4B10AE1A704F4B1C704F4B19704F4BF1
:103A100019689143163A0A431A6060221968914363
:103A2000403A0A431A6007F093FF07F019FFC120DC
:103A3000FF21474B80001A588A431A50C522920032
:103A400098588843BF3901439950985841490840D4
:103A50008021C9010143802099509958C00509026D
:103A6000090A0143995080213B48490107F0F0FFC2
:103A700003232200394901940093394808F068F87B
:103A80002C22384905A807F0B3FE05AC61782078F0
:103A9000023406F017FCA642F8D10121002006F0FE
:103AA0002BFD314B314A196803201140A022D2026C
:103AB0000A431A608022196892040A431A6019683E
:103AC0002B4A1140802292030A431A60294B2A4A4A
:103AD000934200D8012008F043F807F011FF07F0E7
:103AE000EFFE287807F06CFF039B1878C0B208F04F
:103AF000A7F807F04DFE2149042008F039F806F038
:103B00001FFE00F0AFF800F009FE00F097FE00F095
:103B100019FA002011B0F0BD00932100174A0420CB
:103B200008F01EF98023DB059C62FFF787FC5BE74A
:103B30004A0AFF1F34F000401C46FF1FB863FF1FF6
:103B4000480AFF1F490AFF1F680AFF1FBCF0004018
:103B500000E100E0FF00FFFF2046FF1FA458FF1F09
:103B60002056FF1FB0BD001114F00040FF7FF8FF8A
:103B7000FFFF9FFF5071FF1F0080FF1F3B000108E8
:103B800070B500252849294A29484D6308CA1B05F4
:103B90001B0DED188242F9D10022264B8B63264B78
:103BA00008211A628022254B9205DA67244BDA68D5
:103BB0008A43DA60234A1278012A03D09A6822499C
:103BC0000A409A600121EE242048E40002686C4318
:103BD0008A430260DA6811208A43DA6007F090FFB6
:103BE000112007F0ADFF112007F022FF184A200C2A
:103BF0000400642390420AD8FA220023D2009042A3
:103C000005D9144B0A21C01807F092FDC3B2124A1D
:103C10001372124BD4801B78002B04D1104B10214F
:103C2000187808F0A5F870BD00000540880505402B
:103C300000060540FF01000000F0004004E100E044
:103C40003CF000404A0AFF1FFFDFFFFF0038004042
:103C5000B70B000030F8FFFFA063FF1FDC65FF1FFC
:103C6000D863FF1F002210B51100112008F088F85A
:103C700010BD0000F8B5002301250826394F3A4C45
:103C80003B62E3681120AB43E360E368B343E36066
:103C900007F056FF112007F033FF112007F0D0FE88
:103CA0004023226829001343236080236268DB02DB
:103CB000134380226360A36807201343A360A368B3
:103CC0002A4A1340A3608023A2689B011343102259
:103CD000A360236C93432364236C2B4323648023CE
:103CE0005B003B62226B224B1A402263626B1A40DC
:103CF0006263A26B1A40A263E26B1340E3631D4A46
:103D0000E3681340E36006F0C7FB2900072006F0D4
:103D1000F3FB8021184A1120536C0B43536407F0C6
:103D20005FFDFD21154B164A89005A508023C7209C
:103D3000626B5B0313436363E36880003343E360B8
:103D4000E368104A1D43104BE5601958114080226A
:103D500012020A431A50802292051A600B4B5E63CE
:103D6000F8BDC04600F000403CF00040FFFFDFFF20
:103D7000EFFFEFFFFFFF7FFF003800400000FF1F55
:103D8000813B0011FF00FFFF00E100E00000054063
:103D900030B503A804880B20002C0ED14968074DCC
:103DA00008784978090201430A20A94205D1012176
:103DB00020001980024B1B7A137030BD192A0000B5
:103DC000A063FF1FF7B5150008AA16884A680F4FB1
:103DD00014785278120222430A24BA4214D10122E2
:103DE000DBB2019200962A0007F0FAFB041E0BD109
:103DF000074B1B68002B07D068782A780002104315
:103E000042425041013098472000FEBD0229000087
:103E10002463FF1F30B5012503790400BFB02B4296
:103E200012D00A49408806F047FF28420CD06A4663
:103E3000074B69465B8D55801380064B60881B7A63
:103E40001371002203F0FEFF3FB030BD1C63FF1F63
:103E50006042FF1FA063FF1F10B50549054806F02B
:103E6000E1FE0421044A054806F09EFE10BDC0464E
:103E70001C63FF1FFFFF0000DCBD00116042FF1F3D
:103E800010B5024804F060FE10BDC046153E00119A
:103E9000062310B5837010330371443B43712A33FA
:103EA00083714433C37100230222012103720E4B3C
:103EB000027041701C8881724472197A0273C17257
:103EC0009A784273DA7882730322C2731A79027481
:103ED0005A7942740C2282749A79C274DB79037520
:103EE0001123C370152010BDA063FF1F10B514204F
:103EF00007F0AEFC124B14220021186007F020FFDF
:103F0000002007F0BDFC012007F0CAFC022007F0EA
:103F100047FE032004F0BCF8042006F0D1F8052089
:103F200003F0FAFA062003F0C7FF072001F088F932
:103F3000082006F019FE092000F06CFF10BDC046F5
:103F40002863FF1F10B507F023FD012007F060FC78
:103F500007F0CEFB002010BD094B10B504009842BD
:103F600005D0012904D12000064906F05BFE10BDF2
:103F70000229FCD1013904F0A5FD0028F3D0F6E7B1
:103F8000FEFF00004E63FF1F30B5012503790400DA
:103F9000BFB02B4218D00D49408806F08DFE284254
:103FA00012D06A460A4B0B491B8813800A235380A0
:103FB000293313716B460922581D07F019FC0022A2
:103FC0006946608803F03EFF3FB030BD4E63FF1F7F
:103FD000FE42FF1FA063FF1F70B50D7A100004AAF8
:103FE0002C00168810221440154220D1002E20D11A
:103FF0000A78022A18D14A68517815780E4A0902BF
:104000002943914205D00D4A914209D01C800A24CF
:1040100004E014220A491A8007F0EAFB200070BD70
:104020000C2208491A80F7E71C800124F6E70824CF
:10403000F4E70B24F2E7C046F3FF0000F4FF0000B2
:10404000A044FF1FB8BE001110B50400074908487E
:1040500006F0E8FD074804F0B7FC0020E40704D5AB
:104060000721054A054806F09FFD10BD4E63FF1F5E
:10407000FFFF0000593F001120BE0011A442FF1FA6
:1040800000B50C4BBFB01A780B4901A800F008FC32
:104090006B4680B25880002809D06A46074B6946B3
:1040A0001B881380064B0022188803F0CBFE3FB01C
:1040B00000BDC0462C63FF1F2D63FF1FFE42FF1F84
:1040C000FE43FF1F00B50C4BBFB01A780B4901A887
:1040D00001F0FEFD6B4680B25880002809D06A4688
:1040E000074B69465B8D1380064B0022188803F04E
:1040F000A9FE3FB000BDC0465663FF1F5763FF1FB8
:10410000A442FF1FFE43FF1FF7B50E00377A1C00C5
:1041100008AB11003D001A8820231D401F423CD1EE
:104120003378022B3BD173681F785B781B023B43CB
:104130001E4FBB4208D01E4FBB4214D01D4DAB4298
:1041400021D00A252800FEBD002A2AD1142C2AD805
:104150002200F06807F04CFB174B1C70012CF1D9C2
:10416000FFF7B0FFEEE7002A1BD1202C1BD822005E
:10417000F06807F03DFB114B04211C70104B1878C0
:1041800007F0F6FDDEE7E3B20124009201940A0095
:10419000310007F025FA0500D4E70825D2E701250C
:1041A000D0E70B25CEE70D25CCE7C046F3FF000096
:1041B000F4FF0000022900005663FF1F2C63FF1F5D
:1041C000D863FF1F10B5024804F0BEFC10BDC04606
:1041D000893F001170B5160004AA148805AA157845
:1041E0004A685078117800022A4A08438018052846
:1041F0004BD807F075FC03131E29343F0720032C0E
:104200000BD80422121BAA4200D92A0022491A8084
:104210003000091907F0ECFA002070BD0720112CBE
:10422000FBD81222121BAA4200D92A001B491A806D
:10423000EEE707200E2CF0D80F22121BAA4200D95D
:104240002A0017491A80E3E70720032CE5D8042247
:10425000121BAA4200D92A0012491A80D8E7072067
:10426000032CDAD80422121BAA4200D92A000E49D4
:104270001A80CDE70720032CCFD80422121BAA42B4
:1042800000D92A0009491A80C2E700220A201A80B0
:10429000C3E7C046DCD5FFFF6BBE00117463FF1F90
:1042A0005BBE001156BE001151BE00114CBE001184
:1042B00010B50D21024A034806F076FC10BDC04639
:1042C00040BE00111443FF1F37B5002000F0CCF8AA
:1042D000204D214BEA89287C9A422AD1042201A947
:1042E00000F076F9040000F033F9002C30D16B4671
:1042F00099882B68C9BA4B432989184A1B145B1843
:1043000053806B46D9886B6849BA89B24B43698937
:104310001B0C5B181248191C1BB2834200DD011CE8
:104320000B0400D5002113889180013313802000F5
:104330003EBD0223002101AA00F01CF96A460400D8
:1043400002230121287C063200F014F90443CAE755
:104350000124ECE78863FF1F83050000A063FF1FB3
:104360000F27000037B5012000F07EF81F4D07220F
:104370006946287C00F02CF9041E33D16B461B786B
:104380007F2B2FD800F0E4F86B46D878F023020496
:104390001B031A406B469B8815495BBA9BB21A43B4
:1043A0002B68000953432A891B0C9B184B806B46D2
:1043B0005A789B7812031B011A436B6802435343DC
:1043C0006A891B0C9B180B481A1C1BB2834200DD28
:1043D000021C130400D500220B888A8001330B8055
:1043E00020003EBD00F0B4F80124F9E78863FF1F08
:1043F000A063FF1F0F27000010B50F4C237C002B7C
:104400000CD0382B0BD1012000F02EF8CC22AC219F
:10441000207C920100F028F900F09AF810BD074BBB
:10442000E2899A42FAD1012000F01EF80021207C96
:1044300000F0FAF8F0E7C0468863FF1F830500002C
:1044400010B5084B1A7C002A09D05B69002B06D0F6
:104450009847041E01D0FEF7D3FD200010BD0124B3
:10446000F9E7C0468863FF1F70B5002106001620DB
:1044700006F07EF80121152006F07AF807F098FA88
:104480000400092007F0DCFA00222B4B2B4DDA66E2
:1044900061321A6019685B3A9143002E28D0023AC3
:1044A0000A431A60AC4209D10A22DA6107321A6261
:1044B00000221A639A630132DA6370BD204A944283
:1044C00003D11E22DA610532F1E71E4A944203D17C
:1044D0003022DA610632EAE71B4A944203D14322D2
:1044E000DA610832E3E7194A9442E1D16922F7E739
:1044F00002220A431A604622AC4203D0104A944278
:1045000004D194225A6106329A61D1E70D4A94424D
:1045100001D1E622F6E70C4A944204D13422FF325C
:104520005A610D32F0E7094A9442C1D1E6225200A5
:104530005A610A32E8E7C046005000400024F40007
:104540000048E801006CDC020090D00300D8B805F8
:1045500010B50024064B0920DC6607F0F1FA2100B3
:10456000162005F099FF2100152005F095FF10BDDC
:1045700000500040F8B51C000023134D0F00EB66FF
:104580006860160007F00CFC01238022EB66230014
:104590002F615200013B08D207F0BAFA08200B4AFB
:1045A0001168002C03D12000F8BD2A61F2E72B6FBF
:1045B000034203D02B69013C3370013613685B1A48
:1045C000032BEED90124EEE7005000406008FF1FE6
:1045D000002370B5124D1400EB6668600E0007F002
:1045E000DFFB01238022EB6623005200013B08D24F
:1045F00007F08EFA08200B4A1168002C03D1200026
:1046000070BD2A61F2E72B6F034203D02B69013C96
:104610003370013613685B1A032BEED90124EEE7E1
:10462000005000406008FF1F002370B50C4C0D00C7
:10463000E366606007F0B4FB0123E366256107F0E1
:1046400067FA8020074A80001168636B034205D136
:1046500013685B1A032BF8D9012070BD0020FCE71A
:10466000005000406008FF1F002370B5134C0E007F
:10467000E3666060150007F093FB0123E3662661A3
:104680000F33626B1A42FCD02B0A23611023626B3A
:104690001A42FCD0EDB2256107F03AFA8020084AB0
:1046A00080001168636B034205D113685B1A032B0A
:1046B000F8D9012070BD0020FCE7C0460050004042
:1046C0006008FF1F002370B5124D0C00EB66686098
:1046D000160007F065FB0123A619EB660F33B44201
:1046E0000ED107F015FA80200B4A800011686B6B21
:1046F00003420CD113685B1A032BF8D9012070BD5B
:1047000022782A616A6B1A42FCD00134E7E7002064
:10471000F5E7C046005000406008FF1F10B5084C88
:10472000E368002B08D1074B1B685B045B0C0A3362
:104730006360054B1B68236007F032F9A06010BD71
:10474000C863FF1FC8F00040CCF0004010B507F070
:1047500027FB0F4B996A9A6A8A42FBD10D4C62681B
:10476000A0688A18121A531E884200D31300A16051
:104770002168DA0B52185B0407495B0C6360226006
:104780000B60064B1A6007F0C3F9206810BDC046E5
:1047900000F00040C863FF1FC8F00040CCF00040AC
:1047A00070B51D4C23793F2B01D93F2323711B4B3F
:1047B00022791A701878C0B206F0CAFF1823184977
:1047C000184A0B80184913800B805380A37917492E
:1047D00080200B800C21938001334B430001191C76
:1047E000834200D9011C124BD18019806379002BC0
:1047F00001D101336371237A012B01D80223237283
:104800006279237A0B4853430A21584306F090FFFC
:10481000094D286070BDC046BC63FF1F480AFF1FDA
:10482000FC43FF1FC845FF1FFA43FF1FA865FF1F7A
:10483000F843FF1F71020000AC63FF1FF8B51021A1
:104840000020FEF7C3FD114C011E114D09D10C22B1
:10485000104BC1CBC1C4280007F072FAFFF7A0FFCC
:10486000F8BD0C2220000C49FEF784FD0C2802D074
:10487000084B43CB43C40C2228000849FEF77AFDBD
:104880000C28EBD00C220021E5E7C046BC63FF1FDB
:104890008863FF1FACBE0011FC0C0000F50C00008B
:1048A000F0B5002504000E0085B0AA426AD04B1C6A
:1048B000087801934B788978377909021943F3789E
:1048C0003F061B040B431F43039720706570262887
:1048D00000D192E01CD8102812D807F021F94D0021
:1048E00000013300330033009800A6009F0033001E
:1048F0003300330033003300330033003300E6006D
:10490000232800D1C0E025285FD0FF2363709BE0FF
:10491000602800D1A3E00CD8552836D056284ED0B8
:104920003328F2D109229849601C06F061FF0A255C
:1049300028E0722800D189E0DC2800D1E8E0712865
:1049400000D179E0DB2800D0FDE0042ADDD9102574
:10495000052A05D0551F2A003800711D06F048FFB2
:1049600005223100200006F043FF2A003900601DB7
:1049700006F03EFF053505E00C222000834906F0D5
:1049800037FF0C25280005B0F0BD013A804D0C2AF8
:1049900013D8002A0AD02800019906F029FFFFF752
:1049A000FFFE0C2228007B49FEF71EFC29000C228A
:1049B000601C06F01DFF0D25E4E70C22EBE7744DAB
:1049C000754B2A0043CB43C2E9E7013A734D0C2AE9
:1049D00011D8002A08D00199280006F009FF0C22FE
:1049E00028006F49FEF700FC29001322601C06F026
:1049F000FFFE1425C6E70C22EDE7684B29001322C1
:104A000018001D0007F09CF9FEF7FAFAECE7052202
:104A10006449601C06F0ECFE0625B3E712226249E9
:104A2000601C06F0E5FE1325ACE708225F49601C18
:104A300006F0DEFE0925A5E77178F72900D964E7BD
:104A40005B4B188801F0A0FD02259BE7594B012A1A
:104A500003D072785A706270F6E75B7856E7013AD5
:104A6000554D062A0ED8002A05D00199280006F0D7
:104A7000BFFE01F005F829000622601C06F0B8FE12
:104A800007257FE70622F0E7042A04D94B4D2F6063
:104A900006F086FFA860FFF759FE0422039003A9E1
:104AA000601C06F0A5FE05256CE7454D062AE2D9F7
:104AB00006222800019906F043FE0028DBD00622DA
:104AC0000199280006F094FE06223E492800FEF7D0
:104AD0008BFB0123374A51780B435370CBE7931E6E
:104AE000394E1A2B0CD8551E2A000199300006F0B9
:104AF0007FFE3649AAB23000FEF776FB00F048F997
:104B0000334B31001D78601C6A1E06F071FE39E7D8
:104B1000022A00D8F9E67378BFB26370B378A37045
:104B2000032A05D0033A390092B2F01CFEF75CFB71
:104B300010223900E01CFEF71DFCC51C002800DB1C
:104B400020E7607080E7DA2800D0DEE6042A00D88B
:104B5000DBE6082A15D9B37972791B021343F2797F
:104B600012041A43337A1B0613433B603B68052249
:104B700031002000039306F03BFE0422601D03A9D0
:104B800056E7FE236370F1E7A063FF1FB8BE001174
:104B9000BC63FF1FFC0C0000ACBE00118863FF1F4C
:104BA000F50C00009463FF1F7463FF1F3C45FF1F5B
:104BB000FE43FF1FB863FF1F9944FF1FC863FF1F19
:104BC0006509FF1FADAC0000BB65FF1FAEDE000036
:104BD000B965FF1F70477047020010B5094B0A32D4
:104BE000094C92B2DA815A8298811882207802F0B8
:104BF00031FB0422054B012120781A7007F0B8F828
:104C000010BDC046C644FF1F0666FF1F0566FF1F96
:104C1000013870B5042809D806F062FF0309250899
:104C20001200214B0221187807F0A2F870BD1E4B2C
:104C30000821187806F01CFF00221C4B1A72F5E7B9
:104C400000241A4B184D1A68082128781C8106F098
:104C50006FFF2100287807F03BF8012000F048FEA4
:104C600000F00EFFE2E7104B0821187806F000FF75
:104C70000F48FFF70DF90F4B0F4A9B7900209380E7
:104C80000E4A13808022094B52001A8100F030FE38
:104C900000F0F6FE0A4B5B78002BC7D0094A136080
:104CA00007F056F8C2E7C046D863FF1FAC63FF1F8A
:104CB0000744FF1FBC63FF1FC845FF1FA865FF1FF8
:104CC000B863FF1F34F0004010B5012909D1054B2E
:104CD0001B78002B05D02622034B04485A72FFF79D
:104CE0007BFF10BDDC65FF1FAC63FF1FC409000024
:104CF0000300F0B50A4D8E18B14202D1520080185F
:104D0000F0BD0C782F6824093C5D0F271C700C78CF
:104D100001313C402F683C5D5C700233ECE7C046DB
:104D2000F443FF1F0D22114B10B51A700C23104CC9
:104D300010492370093A033B0F48637006F058FD91
:104D40002D2301220D490E48A371FFF7D1FF012247
:104D50000C49FFF7CDFF01220B49FFF7C9FF0022E5
:104D60000A491000FEF740FA10BDC046D865FF1F83
:104D7000B965FF1F6BBE0011BB65FF1F6709FF1FF1
:104D8000C065FF1F6609FF1F6509FF1FAEDE00003B
:104D900010B51D2207480849FEF7ECFA002805DD8A
:104DA0000922064B013018705A7010BDFFF7BAFF88
:104DB000FBE7C046BB65FF1FAEDE0000B965FF1F05
:104DC00010B5114B1A781870002A0ED000280BD19C
:104DD0000E4B1A78062A07D85423D340DB0703D595
:104DE0000B4B187802F036FA10BD0028FCD0074BA8
:104DF0001B78012B02D0033B022BF5D8044B012179
:104E0000187806F0B5FFEFE7DC65FF1F0566FF1FAA
:104E10000666FF1FF8B5544E544A554930700820B5
:104E200005F06CFC0121022005F066FB022005F074
:104E30004FFC0121002005F05FFB002005F048FC3D
:104E400000F0EAFEFEF7DCF806F062FC03224949B6
:104E50004948FFF74DFF2D24030004221C704749E9
:104E60000130FFF745FF30230470454D454C43703A
:104E700083702E3B062220004349EB87FEF77AFA27
:104E8000062813D0200006F013FD022809D00321C4
:104E9000200006F005FF8D23E3706E3B237119336C
:104EA0006371062220003849FEF79EF9374B1B68D4
:104EB000FC335C64FFF76CFF0020FFF781FF344F89
:104EC000344A0121344B1278387802F085F9334C9A
:104ED000334B00211A783878230002F07DF9012243
:104EE0002178304B01391A7000202F4AC9B205F0E1
:104EF00079FD2E4B9B78552B31D13C222C4B5A728D
:104F00002C4A2D4BAA81EB812A826B82202130789A
:104F100006F006FF0120404205F0B0FD01204042AE
:104F200005F04CFEFFF7C4F9FEF796FF00F094FC85
:104F300001204042FFF788F8012006F0E1FEF7204B
:104F400001F006FB0121307806F012FF307802F004
:104F5000DDFA1A4806F0B4FEFEF78CFEF8BDFA2220
:104F6000174B5201CEE7C046D863FF1FD54B001147
:104F7000C94C00113C45FF1F7463FF1F9463FF1F62
:104F8000C644FF1F6509FF1FADAC00006466FF1F2C
:104F90000666FF1F2644FF1F0744FF1FB965FF1F5A
:104FA000D865FF1FAA65FF1FBB65FF1FB863FF1F02
:104FB000AC63FF1FC4090000CE090000DA63FF1FC5
:104FC0004A1F0000F8B50A0020230D001A401942BC
:104FD00047D04F4B1B78002B40D0FFF7B7FB4D4B12
:104FE0004D4C4E4E99686268737A8A1ADB039A4276
:104FF00002D36160FEF73EFE327A217A531EDBB2A5
:10500000994205D1FFF7F8F9002000F0EDFD0FE01F
:105010009142F9D300232372FFF712FA012000F026
:10502000E3FD3F4F3800FEF733FF390006F040FE46
:10503000637A002B0FD0013BDBB26372002B0AD1E5
:10504000384B9B78552B01D106F082FE6423707992
:105050005843FFF7C1FD237A0133237220206840B3
:10506000F8BD0BB2002B0ADA2F4B187806F0C8FCFB
:10507000002801D006F0CCFC80200002EFE70224DB
:10508000214206D0244B01201A72FFF799FE20001E
:10509000E5E70B071ED5FFF759FB1E4B1E491F4CBA
:1050A00098684A68637A821ADB039A4202D348609E
:1050B000FEF7E0FDFFF7C4F9FFF79EF9012000F0CD
:1050C00093FD00F0E3FB2368DB0701D5FFF77AF8D7
:1050D0000820C4E71024214206D00D4B1B78002B7A
:1050E000D5D1FEF7CDFED2E70124214207D00F48EB
:1050F00000F06AF806F094FC00F0EAFCC7E704242C
:10510000080020402142ABD0FEF7BAFFBFE7C046FF
:10511000DC65FF1FC863FF1FAC63FF1FBC63FF1F7D
:105120000744FF1FB863FF1FD863FF1FEC43FF1F37
:10513000F0B51B4B1B4F1B883A8804001A4E1B4DC1
:1051400085B09A420DD832889A420AD3184B1A88F1
:105150002B889A4205D1174A174B12881B889A420E
:105160001BD0052001F04AFA3B8802AA138033883D
:10517000019053802B88114D93800F4B02A91B88FF
:10518000D3800F4B2A78188802F066FF0D4B082158
:105190002878019A1C7006F06BFD05B0F0BDC04682
:1051A000A665FF1FFC43FF1FFA43FF1FA865FF1FF3
:1051B000A465FF1FA265FF1FF843FF1F0666FF1FC0
:1051C000FE43FF1FA065FF1F13B50C4B1C78002C7E
:1051D00011D1002801D00A4B18600A4A0A4B1178F5
:1051E0000A4A10780A4A01920A4A0092002205F0FF
:1051F000F1FA200016BD1124FBE7C0460566FF1F2B
:105200009C65FF1F0466FF1FF465FF1F0666FF1FF6
:10521000E065FF1FE465FF1F10B5064B12201B78E9
:10522000052B06D1044B13221988044B187801F082
:10523000C1FB10BD0566FF1FFE43FF1F0666FF1F73
:1052400010B500240122114B52421870104B1C70F3
:10525000104B1A8002F05AF904220F4B21001A70E9
:105260000E480C3206F0CCFC102221000C4806F04F
:10527000C7FC07220B4B1C600B4B1C700B4B1C70AC
:105280000B4B1A700B4B1C7010BDC0460666FF1FFF
:105290000566FF1FFE43FF1F0466FF1FF465FF1F27
:1052A000E465FF1FE065FF1FB865FF1FB765FF1FBF
:1052B0000044FF1FB665FF1FF8B5174C06002578A0
:1052C00006A814240078052D23D1B41F134FA5B2CE
:1052D0001824BD421DD88D1FADB2BD4219D8FA2584
:1052E0006D00AA4215D21D000D4F0A3DADB2BD4260
:1052F0000FD80C4C26800C4C21800C4900240A80CD
:105300000B4A1380FFF714FF0A4B0421187806F0AC
:10531000AFFB2000F8BDC0460566FF1F790C0000FA
:10532000750C0000FC43FF1FFA43FF1FA865FF1F19
:10533000F843FF1F0666FF1FF0B50BB20D0089B0E2
:10534000002B00DB70E1A44E307806F059FB041E00
:1053500050D00378A22B00D122E1D02B1AD0912B70
:1053600045D143780E2B42D19C4B82889A423ED144
:105370009B4A83681278052A39D1032018567F2862
:1053800035D0984B1B68002B31D05B68002B2ED09A
:1053900098472CE08078072829D806F0A1FB04283C
:1053A000183F3F74A8D86378002B0CD101218C4B97
:1053B00019708D4B1A78002A5BD08C4B307801F035
:1053C0000BFF002855D00722854B1A7051E06178F9
:1053D0000029F8D1E378002B11D0854A854B12784B
:1053E000307801F0F9FE60706378002BEBD120007B
:1053F00006F00EFB80200002684009B0F0BD784B3B
:105400001B78022BF3D00121307806F059FB0028DD
:10541000EAD10121307806F0ABFCE5E76378002B98
:10542000D1D16F4F032807D13B78052B02D101332F
:105430003B701EE00223FBE76F4B1A886F4B029311
:10544000002A0BD01B78002B03D00121307806F006
:105450000FFC3B78062B04D1013BE9E7029B1A7055
:10546000F7E7042B41D10121029B3078197006F037
:105470007FFC5C4B1B68002BB9D01B68002BB6D09F
:10548000574A107884E76378554F002B27D10622BE
:10549000211D5B4806F0ACF962895A4B5A491A80C3
:1054A000A2895A4B1A80E3890B800521397058492B
:1054B0000A80584A1380228A574B1A80574B1B7810
:1054C000012B09D11F2001F099F8FA2292004243E2
:1054D0000421307806F0CCFB0022484B75E7312BD5
:1054E00000D070E70022454B1A700323A0E7062284
:1054F0000021434806F084FB0023454A0421138021
:10550000444A30781380444A138006F0B1FA0821E7
:10551000307806F0ADFAA379083B5A425341304A3D
:1055200003331370304B1B78002B06D0334B30788D
:105530001A78002A06D001F08DFE0122314B52422A
:105540001A8096E70121197006F012FCF5E7082190
:10555000307806F08DFA6378002B00D047E72C4BAB
:105560002D4F0293E388029A04211380294B30784F
:1055700003932389039A138063893B8006F0A0FA82
:10558000002800D033E7264B1B68002B00D12EE704
:10559000039902983A88098800881B68984726E78B
:1055A0004379132B00D022E70389012B0AD11D4B2D
:1055B0001B78022B06D10821307806F059FAFFF744
:1055C0002BFE14E7052001F019F8082102003078BD
:1055D00006F04EFB0BE7C0460666FF1F05140000F1
:1055E0000566FF1F9C65FF1F2644FF1F0744FF1F22
:1055F000D865FF1FB965FF1FDA65FF1FDC65FF1F58
:10560000AB65FF1FFE43FF1FB265FF1FB465FF1FA1
:10561000A665FF1FA465FF1FA265FF1FAA65FF1FE8
:105620009865FF1FA065FF1F8020C001014200D0C8
:10563000E2E6CB0731D5324B1B78002B1DD0314E23
:1056400005AC3378052B1AD1023B23702E4B210079
:105650001B7823722D4B1B7863722D4B187801F049
:105660005FFD002809D007202A4B30701B68002BF3
:1056700003D01B68002B00D098470120BCE60E2009
:10568000254B06221B7825492370254B1B78637018
:1056900002ABC01806F0ACF8D8E7022308001840A7
:1056A000194209D0174B1B78052B03D11D4B1888C5
:1056B00006F0E6FA02209FE60424214203D0FFF719
:1056C00037FD200098E6082308001840194200D151
:1056D00093E6154B1C78012C03D0022C0DD008202A
:1056E0008AE6124B124A134913481B88128809880C
:1056F00000880094FFF7E0FDF1E7FFF78DFDEEE78E
:10570000DC65FF1F0566FF1F0044FF1FB665FF1F16
:105710000666FF1F9C65FF1FB865FF1F0144FF1F42
:10572000B765FF1FFE43FF1FA065FF1FF843FF1F64
:10573000A865FF1FFA43FF1FFC43FF1F10B502A817
:1057400004880B20002C10D1496808784978090298
:1057500001430C48814209D1022119800A4B598822
:105760001170DB7800205BB2537010BD074C0A202B
:10577000A142FAD102211980034B998811705B79FB
:10578000F0E7C0466E2A0000A063FF1F6F2A0000EA
:10579000F7B5150008AA16884A680F4F1478527892
:1057A000120222430A24BA4214D10122DBB201922E
:1057B00000962A0005F014FF041E0BD1074B1B684E
:1057C000002B07D068782A780002104342425041EB
:1057D000013098472000FEBD022900001866FF1F17
:1057E00030B5012503790400BFB02B4227D01549FD
:1057F000408805F061FA28420DD06A46124B69468E
:105800005B8D138002235380104B5B8893806088EC
:10581000002202F017FB0E49608805F04DFAC00720
:105820000DD56A460B4B69461B88138002235380B3
:10583000064B9B8893806088002202F003FB3FB0F8
:1058400030BDC0461066FF1F2844FF1FA063FF1F26
:105850000866FF1F8244FF1F10B5074C0749200050
:1058600005F0E0F92000064905F0DCF90721054ABA
:10587000054805F099F910BDFFFF00001066FF1FF5
:105880000866FF1F38BF00112844FF1F10B50248EB
:1058900003F05AF910BDC046E157001170B55F25FD
:1058A000082607498400CA788B7840012A40B34310
:1058B0003440A843234302438B70CA7070BDC04676
:1058C0009944FF1F010043B204205A0002409B008C
:1058D0000C3003401A43152310B5044CE07898436C
:1058E000143B0B4018430243E27010BD9944FF1F64
:1058F00010B5054B082419790A00A243002801D0ED
:1059000022000A431A7110BD9944FF1F10B5054BC0
:105910004024D9780A00A243002801D022000A437B
:10592000DA7010BD9944FF1F0821F8B5324D334B92
:10593000AE7804000E40AE70984204DD67232B70F1
:10594000473B6B70F8BD2E4B984203DAE0232B7077
:105950003A3BF6E700232B706B7083B21A0029489C
:105960005F3292B2284F82422CD9002C03DA5B427C
:105970001CB204232B70053420B20A2105F0D8FE96
:1059800004B2FA239B009C4232DB08232A7813439B
:105990002B706421200005F0CBFE0A2100B206F036
:1059A0006FF809B22A787B5C13432B700A21200020
:1059B00005F0BEFE0A2100B206F062F809B27B5C77
:1059C0006A780AE06970002CDBDA5B421CB20423BF
:1059D0002B70F3226B78092CE8DC13436B700A21DF
:1059E000200006F04DF809B27B5C1E43AE70A9E7BB
:1059F000632CCEDCEDE7C0469944FF1F1B4E000030
:105A00001DFCFFFF2A08000062BF00110823F7B544
:105A1000194FCD003E7904001E403E71EDB263285F
:105A200006DD5F3333433B7120231D437D71F7BD9A
:105A30000300093305DA20235B4233433B71A6237D
:105A4000F3E70E4B019300280BDA0423444224B2FF
:105A50003B710A21200006F013F8019B09B25B5C40
:105A6000E3E70928F5DD0A2105F062FE019B00B29B
:105A70001B5C1E433E71ECE79944FF1F62BF00119F
:105A800070B50F4B1B78002B18D00E4E0E4D062212
:105A90003100280005F054FE00280FD00622310006
:105AA0000A4C280005F0A4FE0120FEF7DDFC0722C9
:105AB00021003E20FEF706FEFEF74AFD70BDC046FF
:105AC0002366FF1F9944FF1F1D66FF1F1C66FF1FF3
:105AD000E622402110B50A4B1A70403A5A703E3205
:105AE0009A70DA780A40DA70082219791140053A7A
:105AF0000A431A71F3225A71FFF7C2FF10BDC04664
:105B00009944FF1FF8B51C4B3C21186805F060FF55
:105B10003C21040006F03CF820000F003C2105F079
:105B200057FF182106F034F800230E00134C0A2109
:105B30002370300005F04CFF114D0A212B5C300022
:105B4000637006F025F840226B5C2679A370E37839
:105B500038001340E37008230A211E4005F038FF87
:105B60002B5C0A211E433800267106F011F86B5C8D
:105B70006371FFF785FFF8BDC863FF1F9944FF1FDE
:105B800062BF001110B5164C0A210223E05E05F039
:105B9000CFFD00B2FFF7C8FE0423E05E642105F0EC
:105BA000C7FD012100B2FFF731FF237A0024132241
:105BB00020009A426041C0B2FFF7A8FE0320FFF721
:105BC0006DFE2000FFF77EFE064B18780538434235
:105BD0005841C0B2FFF78CFEFFF752FF10BDC04620
:105BE000A063FF1F0566FF1F094B10B51B689B07CD
:105BF00008D5084A1378591C1170DB0704D5FFF744
:105C000081FF10BD0028FCD0FFF7BCFFF9E7C046BC
:105C1000BC63FF1FB863FF1F002010B5FEF724FC14
:105C200010223E200549FEF74DFD0023984200D189
:105C30003E33034A1370FEF78BFC10BD52BF0011B8
:105C40002366FF1F0200F0B501270A480A4E5118CB
:105C50008B1A002B00DCF0BD08241578430868403F
:105C600038404000805B013C58406D08002CF5D165
:105C70000132EDE7FFFF000072BF0011F0B5002513
:105C80000F269D4200DBF0BD4C5D070944403440C7
:105C9000A400A05801357840F3E70000F0B589B0C2
:105CA0006A460D000B000F27110010351C780133D8
:105CB000260024093E40167054700232AB42F5D1E2
:105CC0002023024AFFF7DAFF09B0F0BD78BF0011C8
:105CD000F0B54E780B7889B036020C0017000190B1
:105CE0001E43012A61D9954B9E4200D877E00133CB
:105CF0009E421CD1062A17D1CA788B7812021A4309
:105D00000B791B0413434A7912061A438C4B5A61D0
:105D100000221A705A808B4A5A608B4A9A608B4ACA
:105D2000DA60002009B0F0BD88225205EEE7884B0A
:105D30009E423CD182498B78002B00D0F6E00C2AA1
:105D400031D10F22A3789343E278120213432279D0
:105D5000120413436279120613434B60E279A0796F
:105D600012020243207A00041043627A12060243B0
:105D7000CA60E27AA07A1202024376484A818342DC
:105D800008D804236E49142201980B7005F030FDE9
:105D90001420C7E71201D21889235B059A42F0D874
:105DA00001238B70BDE7022AFAD00523EAE76A4A8D
:105DB00001239642E6D1FFF72FFA052F0CD9E3789D
:105DC000A2781B021343227912041A4363791B063B
:105DD0001343624A0393136005F0BAFFA1E7584DDD
:105DE0002B78002B9DD1AB78002B00D1A0E02B8924
:105DF00001339BB20093B34200D091E0132AD4D96F
:105E0000CF7C8B7C3F02122120001F43FFF71AFF3B
:105E1000874200D08EE0002E3DD1E378A2781B02AD
:105E200013432279E96812041A4363791B0613436A
:105E300003930A228B4212D1FF23A370E3702371D4
:105E400063716B89002B09D1E37B227C1B02120456
:105E50001343A27B13431B0901336B8100226B891F
:105E6000002B8ED0002A67D1686837013818000BE4
:105E70006B6900030390984205D9686105F058FDED
:105E8000EB780133EB7068681022A11C381805F01C
:105E900077FD2E8145E76F89009A7B1E9BB2934266
:105EA0003AD1E278A37812021A43237905A81B0499
:105EB000134362796C6812061A43EB6800920392EE
:105EC000211D0C22049305F093FC0120260004A957
:105ED00040421036FFF7E2FE013F012F17D1009A32
:105EE0000B232861824200D04CE704221C49200089
:105EF00005F046FD042203A9686805F0C9FCE968BD
:105F0000039AFF23914200D13CE7F73B3AE7310087
:105F1000FFF7C4FE1036DFE70923B742A4D831E704
:105F2000009BB34200D9FCE607232BE7022329E7B5
:105F3000032327E7062325E70A2323E7FFFE0000C4
:105F4000A044FF1F00000111FFFF00005048593618
:105F500001FF0000FFFF001102FF000034F00040CD
:105F6000AC44FF1F10B5034C0B000122210000F0D0
:105F70006BFA10BD256100110B8870B506000D008D
:105F80000224162B11D92B000322094900F05CFAD8
:105F9000041E0AD1074B2A881B88191C934200D97A
:105FA000111C300089B200F0EFFA200070BDC0462D
:105FB000516100117E66FF1F10B54A780400013A56
:105FC0000B000220012A07D80A78002A04D00522F3
:105FD0002000024900F038FA10BDC0467F61001170
:105FE0000A7810B50B0004000220002A04D0072212
:105FF0002000024900F028FA10BDC0462B620011B3
:106000000A7810B50B0004000220002A04D00922EF
:106010002000024900F018FA10BDC046916200113C
:1060200010B5034C0B000B22210000F00DFA10BD3F
:10603000C162001110B5034C0B000D22210000F0CD
:1060400003FA10BD3363001110B5034C0B000F228F
:10605000210000F0F9F910BD8D6300110A7810B528
:106060000B0004000220002A04D011222000024963
:1060700000F0EAF910BDC0469D630011002310B581
:106080001322190000F0E0F910BD000010B5034C18
:106090000B001722210000F0D7F910BDEF630011AB
:1060A000002310B51922190000F0CEF910BD000030
:1060B00010B5034C0B001B22210000F0C5F910BDE8
:1060C00029640011F7B584890D0006000121002C18
:1060D00022D000238268D3561778002B1EDA0C2CAE
:1060E0001AD90C3CA4B2131940880093230002F083
:1060F00086FE431E984101307B06DB0F6B703F2309
:10610000013C1F40A4B22870AF70AC80002C07D0B7
:10611000B3680133AB6000210800FEBD0020EBE74F
:10612000AC60F8E70B7803704B8843704B881B0A10
:1061300083700B79C370042070470420022B06D1B2
:106140000020537811781B02009A0B43138070478C
:106150000B8803700B881B0A4370022070470420D1
:10616000009983420AD1537810781B0203430B80B5
:10617000D37890781B02034300204B807047F8B51A
:106180000D004B7801240021461C03702B788B42B4
:1061900001D82000F8BD6B78B01C4F1C012B10D12A
:1061A000890069184B88022233704B88B9001B0A9A
:1061B0007370691805F0ECFD04360434A4B2F9B22A
:1061C000E4E7122359436B185A88043132705B8814
:1061D00010221B0A7370691805F0DAFD12361234AA
:1061E000ECE770B5049D14001E00052B01D80420B7
:1061F00070BD637812781B0213432B80E378A2787A
:106200001B02134302226B802A71211D681D063E6A
:1062100005F0BEFDB2B22A81F02AE8D82800A11DFF
:106220000A3005F0B5FD0020E2E7002310B50A783A
:106230009A4201D8900010BD9A008A185488013300
:1062400004705488DBB2240A447094888470928865
:10625000120AC2700430EAE710B51100029C062B46
:1062600004D004201022142B01D010BD0222227170
:106270004B7808781B0203432380CB7888781B0275
:10628000034363800431601D05F082FD0020ECE7CC
:1062900010B50C788B7804315C43E4B203702200B3
:1062A000013005F075FD601C10BD0420022B06D1E5
:1062B0000020537811781B02009A0B43138070471B
:1062C00010B50C000A88023105F062FD208810BD6F
:1062D00070B504000D0004981100012B01D80420B2
:1062E00070BD167852781202324302800200F832F2
:1062F00055701470E825002C00D10C35023B9AB281
:106300004280AA42EBD80231043005F041FD002062
:10631000E6E70420009983420AD1537810781B02E3
:1063200003430B80D37890781B02034300204B80FB
:10633000704710B50C000A88023105F029FD20884D
:1063400010BD000070B501211E000420049C0E4009
:106350000B4218D1CB40DDB28D4214D90A49DBB2D1
:10636000098899420FD32300F6331D70330058007B
:1063700011184978165C0902314301332152D9B210
:106380008D42F4D8002070BDC044FF1F10B50C0032
:106390000A88023105F0FCFC208810BD10B50C788D
:1063A0008B7804315C43E4B203702200013005F0C5
:1063B000EFFC601C10BD10B511000298032B01D832
:1063C000042010BD14785278043B1202224302804C
:1063D000CA788C781202224342809AB28280F22AD2
:1063E000EED80431063005F0D3FC0020E9E710B503
:1063F0000C000B8803700B881B0A43704B8883705A
:106400004B881B0AC3708A880430063105F0C0FC33
:10641000A088043080B210BD0420012B03D10020DD
:106420001378009A1370704710B50C000B88037036
:106430000B881B0A43704A880230043105F0A8FC1F
:106440006088023080B210BDF0B589B003931E4B56
:10645000029242000700D05A019102F020F8132561
:10646000061E2DD0029B01240370019B002B04D03B
:10647000001903999847001984B26B461B7A5BB2E6
:10648000002B0FDA1021380002F01CFB1925002820
:1064900013D130003219E1B202F066FC051E0CD1B6
:1064A0000C34A4B2042304AA380005A993800696EC
:1064B000948101F0AFFD051E02D0300005F040FAD6
:1064C000280009B0F0BDC0467C66FF1F70B505000E
:1064D0000C0000280CD00020814209D0102220009E
:1064E000044905F055FC01202B7823736B78637306
:1064F00070BDC046B8BF0011F0B506000D00170012
:106500001C0085B002291BD00020102907D1022BC6
:1065100007D0102B03D115E00020102C08D005B0B7
:10652000F0BD69463800FFF7D1FF2A0069460BE04D
:1065300069463000FFF7CAFF22006946380004E0D0
:10654000022BE9D12A003900300005F079F9E6E79D
:10655000031CF72800D9F723032008499AB2013A0F
:106560000B80D317034006499B189B100B80D30F59
:1065700004499B185B100B807047C046C444FF1F42
:10658000C244FF1FC044FF1F034B1B888B4202D332
:10659000024B4000C1527047C444FF1F7C66FF1F7E
:1065A000014B4000185A70477C66FF1F1722014BB1
:1065B0001A8070477C66FF1F70B505000E2005F03D
:1065C00007F9041E13D0D023037000230622837022
:1065D00007494570033005F0DBFB064B2100DA8AE2
:1065E00062811B7E2373044B187805F039FA70BD65
:1065F0009866FF1F8866FF1F1445FF1F262803D8D3
:10660000024B4000C05A70470148FCE7C644FF1FD8
:10661000FFFF000070B506000C00094D1C22002190
:10662000280005F0EDFA074B1E70074B1C7005F0B3
:10663000BFFA0123002801D0002312202B7070BD67
:106640008866FF1F1445FF1FA966FF1F70B5050070
:106650000D4C0800E260A16010220021656005F089
:106660003FFB012803D11021A06802F058FD102241
:106670000021280005F034FB012803D110216068B7
:1066800002F04DFD70BDC0468866FF1F70B5041E48
:1066900005D1002903D006220D4805F079FB0D4BEA
:1066A0001D78012D11D1002C05D102221A7005F0A0
:1066B00057F8280070BD00221A70074B1B78FF2B7B
:1066C000F7D02000FFF778FFF3E70025F1E7C04699
:1066D0009866FF1F8866FF1F1445FF1F030010B553
:1066E000002801D1002010BD00780B4A002803D1FA
:1066F0005988D1821B7913761378022BF2D10023AB
:10670000984200D103331370044B1B78FF2B01D048
:10671000FFF752FF0120E6E78866FF1F1445FF1FC1
:10672000002911D000280CD04B79012803D1402238
:106730005242134303E03F221340032802D00120BA
:106740004B7170474022F4E70800FAE770B5094D35
:106750000100287800280BD0074C0622200005F005
:1067600017FB21002878FFF7DBFF200004F0C8FFAB
:1067700070BDC046A866FF1F8266FF1F00290AD0B1
:10678000012808D13F224B799343C02B03D0403BD3
:106790005A425341981C704770B5174D06002B782C
:1067A000FF2B15D00A2005F013F8041E10D0D023BB
:1067B0000370C83B8370114B11491B784670C3703E
:1067C0000622043005F0E4FA2100287805F048F9A3
:1067D0000C4B1B78012B0DD10B4B1B68002B03D0EE
:1067E0009B68002B00D09847084B04211878084A72
:1067F00005F09EF970BDC0461445FF1FA866FF1F37
:106800008266FF1FA466FF1FD066FF1FD466FF1FAE
:1068100060EA0000014B98687047C0468866FF1F19
:10682000014BDB68186870478866FF1F074B10B57F
:10683000DA68136801331360054B1878FF2803D01A
:106840008021C90105F094FA10BDC0468866FF1F7B
:106850001445FF1FF7B50E0002F0C8F8051E1CD046
:106860000E4B06621F78002F00D10778AB791020FD
:10687000019304F0ADFF041E0FD0D0230380C73B6B
:106880008370019BE91DC3700622043005F080FA75
:1068900021003800E66005F0E3F8F7BD1245FF1F60
:1068A000014B18787047C046A866FF1F054B0028AB
:1068B00005D1054B1A78054B002A00D1014B180071
:1068C0007047C0469866FF1FA866FF1F8266FF1FBD
:1068D000014B58687047C0468866FF1F024B186816
:1068E000431E9841C0B27047AC66FF1F421E0300B2
:1068F0000120152A03D9FF3B5A425341D8B27047B1
:10690000F0B51C0000230E0085B0039002920B70BE
:10691000029A934201D3002019E0E55C5A1CD2B2DE
:10692000002DF8D0029851198142F4DC0233DFB215
:10693000A35C18000193FFF7D9FF002807D0013DA1
:10694000019A0399EBB233708A4202D1E01905B083
:10695000F0BDDB19DBB2DBE710B50C0002F09EF8EE
:1069600003001220002B03D02100588805F028F9DD
:1069700010BD000070B50E4D84006359002B15D07A
:10698000186A002801D005F02BF82B59586A002806
:1069900001D005F025F82B59986A002801D005F0A0
:1069A0001FF8285905F01CF800232B5170BDC04674
:1069B000B866FF1F1C4B70B504000E00150099420D
:1069C0000AD11A4B1B68002B01D1122070BD1B6825
:1069D000002BFAD09847F9E7154B994215D1134B84
:1069E0001B68002B0AD01B68002B07D09847002893
:1069F00004D1104B1C70104B1D70E7E729002000DC
:106A0000FFF7AAFF0028E1D1F3E7080001F0EEFF4D
:106A10000028DAD003780320A342D7D12900300020
:106A200005F0CEF8D2E7C046FEFF0000B466FF1FB7
:106A3000FFFF0000B166FF1FB066FF1FF7B504003F
:106A4000808801F0D3FF0025A84203D00578A088F4
:106A500002F008F81C4E3378002B1FD0AB421DD13A
:106A60001A4B28001978FFF777FF002818D0002369
:106A70003370A3790820A778A688019304F0A8FEB4
:106A8000011E0DD0D0230370CA3B8370019B477059
:106A900086808371280004F0E3FF01E0002DE8D137
:106AA000A0880B4B8200D358002B01D0FFF762FF68
:106AB0001721A088FFF768FDA08801F027FDA088B6
:106AC00001F0FEFDF7BDC046B166FF1FB066FF1FB7
:106AD000B866FF1FF0B587B01D000CAB1B88070020
:106AE00001930DAB1B88142002930EAB1B8816007C
:106AF00003930FAB1B880091049310AB1B88059385
:106B000004F066FE041E1AD0D0230370CB3B4770FE
:106B10008370C670062229000430002D11D005F0C4
:106B200037F9019B21006381029B0098A381039B9D
:106B3000E381049B2382059BA37404F091FF07B0BB
:106B4000F0BD05F05DF8ECE7F7B5009308AB1B88E6
:106B500007000C200D001600019304F039FE041EFE
:106B600013D0280001F042FF00280FD00078D02376
:106B70002370C93BA370009B21002381019B677098
:106B8000A580E680638104F06BFFF7BD014B1878A8
:106B9000EDE7C0461445FF1F13B50400648903895F
:106BA000C2888188C0780094FFF7CEFF13BD000033
:106BB00010B5044C2068002803D004F011FF002316
:106BC000236010BDBC66FF1FA122F0B58188920032
:106BD0004A43384B384F1B6804009B189D22920093
:106BE0009B18827989B01A603B68002B5FD01D78B2
:106BF000324B1B68002B04D05B68002B01D00020B7
:106C00009847260008363100E079FFF7B7FD237D6D
:106C1000E0710200E0780493638A29000393238AD9
:106C20000293E3890193A38800933300FFF752FF97
:106C3000E378002B0BD1E289A379A1880292019617
:106C4000E27928000092012201F0DAFEE0703B6850
:106C5000002B20D0FFF7ACFF194D287800281AD060
:106C6000184B1978FFF778FE002814D02B78E678B7
:106C700008200793A78804F0ABFD011E09D0D0239C
:106C80000370CA3B4670837087808671079804F052
:106C9000E7FE00232B701721A088FFF775FCA08862
:106CA00001F034FCA08801F00BFD09B0F0BD064BEB
:106CB0009DE7C0463409FF1FBC66FF1FD066FF1F5B
:106CC000B166FF1FB066FF1F1445FF1FF8B5070030
:106CD00008000E0001F08AFE041E18D02620FFF7DF
:106CE0008DFC051E00D12578062004F071FD041EE0
:106CF0000DD00021062204F083FFD0232370C23B75
:106D000021006770A370A680E8B204F0A9FEF8BD68
:106D1000F0B585B001930AAB1B78070002930BAB6B
:106D20001B7808000D000092039301F05FFE061E21
:106D300022D0102004F04CFD041E1DD01022002192
:106D400004F05EFF2620FFF759FC002800D13078C0
:106D5000D0232370C13BA370009B21002372019BB1
:106D600067706372029BA580A372039BC0B2E3723B
:106D70000C9BE36004F074FE05B0F0BDF7B50D00A8
:106D8000019001F033FE071E20D00E2004F020FDFC
:106D9000041E1BD02620FFF731FC061E00D13E78D2
:106DA000D0232380C53B0622A370F91DE01C04F00C
:106DB000EFFF019B2A0063810123DD401A401D4043
:106DC000210022736573F0B204F04AFEF7BD0000A3
:106DD000F0B585B0029010000D0017000A9E0393D5
:106DE00001F004FE041E31D0029B002B2ED1039B28
:106DF00002795B0724D5122313430422002E08D105
:106E00000B99002905D10C99002902D10D9900296F
:106E10001AD01A430D9B2271002B00D0C9E0002E1E
:106E200000D1CFE0002D00D0CCE0606A002801D076
:106E300004F0D6FD1C21300004F05AFF606205E02A
:106E400002239A430E33D7E793432371654BBA006D
:106E5000D458002C00D1AAE0002E10D0236A002BB9
:106E600003D11C2004F0F4FC20625E4BBA00D3581E
:106E7000186A002803D01C22310004F089FF0C9B03
:106E8000002B12D0574CBB001D596B6A002B03D14D
:106E9000162004F0DDFC6862BB00E358586A002845
:106EA00003D016220C9904F073FF0D9B002B11D018
:106EB0004C4DBC006659B36A002B03D1142004F07A
:106EC000C7FCB0622B59986A002803D014220D9990
:106ED00004F05EFF380001F089FD051E67D0414BCC
:106EE000BA00D358002B62D01A6A3420002A00D18D
:106EF0001C389A6A002A01D0143080B20B9A002AFA
:106F000001D01C3080B25B6A002B01D0163080B2F9
:106F100004F05EFC041E4AD01822002104F070FE2A
:106F20002620FFF76BFB0190002801D12B780193FD
:106F3000D0232370029B200063700A23294EA37084
:106F4000039BBD00A371AB59A780196A18300029B3
:106F500005D01C22A06004F01BFF200034307359C0
:106F6000996A002907D0030014221433E0600293C9
:106F700004F00EFF02980B9B002B08D003001C228C
:106F80001C330B992061029304F002FF029873599D
:106F9000596A002903D01622606104F0F9FE6B469D
:106FA0002100187904F05CFD3800FFF7E3FC05B020
:106FB000F0BD10220D9B0D991B69A018236204F0EF
:106FC000E7FE2CE70B9B002B00D13FE7012D00D003
:106FD0003CE7606A002801D004F002FD1C210B98F8
:106FE0002AE7C046B866FF1F10B5044C2068002889
:106FF00003D004F0F5FC0023236010BDAC66FF1F36
:107000000B4B07B51A68002A01D100200EBD694656
:10701000531C012012780731FFF772FC0028F4D0CE
:1070200002780123100018401A42EED0EEE7C04665
:10703000C866FF1FF0B51F4F01203B6887B0002BCB
:1070400025D09B78059300F0B3FB002821D00A20BF
:10705000FFF7D4FA04000B20FFF7D0FA164B050017
:107060001E78731E9E413B68F6B2191DD878FFF753
:1070700057FB3B682900DA7A043303929A7901932B
:107080000292009033002000059A04F0B1FD07B091
:10709000F0BDFFF7B5FF002805D00620FFF7AEFAD8
:1070A00004000720D8E70820FFF7A8FA0400092009
:1070B000D2E7C046AC66FF1FA866FF1F70B50A4E38
:1070C000040033780D00FF2B0DD0042004F080FB6A
:1070D000011E08D0D0230370CE3B45708370C4706E
:1070E000307804F0BDFC70BD2445FF1F70B504006E
:1070F00006200D0004F06CFB011E0AD0D0230370A3
:10710000CD3B8370054B44701B688580187804F074
:10711000A7FC002C01D0FFF767FF70BDAC66FF1F16
:10712000F8B5264F06003B680D001124002B05D151
:107130000522234B1B78134202D112242000F8BDF4
:10714000204A10241268002AF8D01278002AF5D0BC
:10715000DB0719D52B789A1E012A1AD80C2004F0C7
:1071600077FB132438600028E8D000230A224370FC
:1071700029000670023004F00BFEFFF75BFF041ECF
:107180000AD0FFF731FFD9E700F012FB0028E1D168
:10719000E4E7002BE2D0D0E70B4B1B78032BCDD1DB
:1071A0001D20FFF72BFA094B18800028C6D0084B8A
:1071B00004211878074A04F0BBFCBFE7AC66FF1F48
:1071C000A966FF1FC866FF1FA866FF1FA666FF1FF0
:1071D000D466FF1F60EA0000F7B50193194B140055
:1071E0001A78052306000F0012201A4221D0012927
:1071F00020D1154B1D68002D1BD002201F2C18D844
:10720000002C02D0019B002B13D0104B1F221E70AC
:107210006E1C0021300004F0F3FC019922003000C4
:1072200004F0B6FD310020002C70002F06D004F0D1
:107230007FFDFEBD064B12201D68DCE704F098FBC5
:10724000F7E7C046A966FF1FC866FF1F2445FF1F5A
:10725000C466FF1FF8B50F4E12243368002B17D0F9
:107260001B780F3C834213D100250B4F0221387845
:1072700004F0FEFB094B042138781D8004F0F8FB74
:10728000074B28001D8033685C7004F031FC04005B
:107290002000F8BDAC66FF1FD466FF1FC066FF1F4D
:1072A000A666FF1F70B5012823D11B4C2388002B35
:1072B00003D01A4A1578002D07D0194B1B68002BF4
:1072C00002D01878FFF7C6FF70BD3B2B02D93C3BBC
:1072D0002380F9E7134E0221307804F0C9FBFA222B
:1072E0002388920002215A43307804F0C1FC2580A3
:1072F000EAE70B4B1B68002BE6D00B4B1B785B07B8
:10730000E2D5084B0221187804F0B2FB0022024BB0
:107310001A80FFF769FED7E7C066FF1FA466FF1F4C
:10732000AC66FF1FD466FF1FA966FF1FF8B51E4D90
:107330002868002803D004F053FB00232B601B4E69
:107340003068002803D004F04BFB00233360184F53
:1073500005243B7818002040234221D0154800F036
:107360002BFA3B78234213D0202004F071FA2860D6
:10737000002813D02022002104F042FC202004F039
:1073800067FA041E306005D02022002104F038FC8A
:10739000002004E0286804F023FB2C601320F8BDD3
:1073A00000F00AFAF4E7C046C866FF1FC466FF1F74
:1073B000A966FF1F1845FF1F10B50A4C23681A1E47
:1073C0000ED0002808D10130587004F091FB00283D
:1073D00005D02368002B02D00021FFF787FE012291
:1073E000100010BDAC66FF1FF7B5274E05003368CF
:1073F0000191181E21D05C78244F012C30D1FFF769
:10740000FFFD002825D02000FFF7F8F804004128F0
:1074100014D91F4B022118781E4A04F089FB1E4B19
:107420003C3C1C80022233685A703B78002B14D1FC
:1074300028000199FFF75AFE0120FEBDFA229200B2
:107440004243002AEED0124B0221187804F010FCBF
:10745000E8E7FFF7D3F80200F3E700233B70EBE720
:107460003B78002BE8D1032004F0B2F9011E08D0CC
:10747000D0230370CC3B457083703368187804F0D8
:10748000EFFAFFF7B1FDD7E7AC66FF1FA466FF1F59
:10749000D466FF1F60EA0000C066FF1F10B51749E1
:1074A000838802008B4220D011D815498B4217D017
:1074B000144900205B1899B2012907D89268117805
:1074C0005A425341D8B2FFF7F9FD012010BD0E4AD0
:1074D00000209B1807229BB29A424041C0B2F5E7B8
:1074E00083681878FFF768FFF0E7836899785A781F
:1074F000090218781143FFF777FFE7E70A20000039
:1075000006200000F8DFFFFFAFDFFFFF014B187020
:107510007047C0462545FF1F10B5064C207001F08E
:1075200041FA207804F07CF90521207800F062FD12
:1075300010BDC046D466FF1F0BB273B50D00002B03
:1075400000DBC4E0884B187804F05AFA041E0ED011
:107550000378912B0FD0A22B00D1A1E0834B187898
:10756000FF2852D0210004F07BFA00284DD1802062
:107570000002684076BD43780F2B76D013D8052BD8
:1075800070D00E2BEAD18088794B98422BD8794B5A
:1075900098421BD8784B9842E0D1A3681878591CC0
:1075A000FFF774F838E03E2BD8D18378032B74D0E2
:1075B0006CD8012B6ED0022BD0D1704B1B68002BE6
:1075C00023D05B68002B20D098471EE06C4BC0187E
:1075D0000C28C3D804F07CF91DC2C2150BC20B0BDA
:1075E0000B3223C23C00674BC0180728B6D8664B45
:1075F0001B68002B09D01B68002B06D02000984781
:107600000AE0A3681878FFF7C7F8200004F000FA32
:10761000ADE7A068FFF762F800289FD0F5E7A36800
:107620001B78002BF1D0554B1B68002BEDD01B684D
:10763000002BEAD0210055489847EDE74F4B1B68D7
:10764000002BE2D01B68002BDFD021005048F3E76D
:10765000504B1B68002BD8D05B68002BD5D0210085
:107660004348E9E7FFF7EAF9CFE780884A4B9842B9
:1076700003D04A4B984200D070E7464B1B68002B62
:10768000C3D05B68002BC0D02100D5E7153B012B90
:10769000BBD963E7FFF798FAB7E7FFF77DFAB4E7DE
:1076A0003F4B1B78042B07D100236A4613800179D6
:1076B000408800F0C5FCA8E7364B1B68002BA4D01F
:1076C0005B68002BA1D00100364898479DE7012454
:1076D00021420AD0294B1B68002B04D05B68002B89
:1076E00001D000209847012043E78B070AD5264B9D
:1076F0001B68002B04D05B68002B01D0200098474A
:10770000022036E70421280008400D4200D131E76D
:10771000254E3388002B21D0013B9BB23380002BB8
:107720001AD1FFF7DBF800280AD0204B1C70164B4B
:107730001B68002B04D05B68002B01D02000984709
:10774000FFF7C6F8694601F001FD6846FEF7FEFF47
:107750001D20FEF753FF308004200AE7024B187803
:1077600004F086F9F8E7C046D466FF1F2545FF1FE1
:107770000E2000000120000009100000CC66FF1F51
:10778000FEDFFFFFAFDFFFFFD066FF1F0C20000012
:107790000B200000B466FF1F0D2000001320000026
:1077A000A966FF1FFFFF0000A666FF1FA466FF1F5C
:1077B00010B501F09BF910BD014B18607047C04631
:1077C000D066FF1F0B880020162B01D8172304203A
:1077D000014A13807047C0467E66FF1F0020704735
:1077E000074A03001188814207D0918800209942FE
:1077F00002D101308000101870470020FAE7C0461F
:10780000DC66FF1FF0B58F7806000D00C7B01E2F95
:1078100015D1FFF7E5FF051E03D10024200047B076
:10782000F0BD00223B003100C078009200F0B2FBB6
:107830000400A81C00F0D3FBFF23EB70EEE7264BFF
:10784000062403931B78FF2BE8D0182FE6D87B087B
:10785000224A013BDB0002929A589446002ADDD06E
:10786000029AD3185B68002BD8D00878002802D180
:107870004B78012B02D10624122FCFD107AFAB8852
:10788000697800976446AA68A047041EC6D1AB7801
:10789000029A5B08013BDB00D318390030005B68BB
:1078A0009847041E0BD1AB78042BB6D0039A310055
:1078B00010782200009700F06DFB0400AEE76A78B4
:1078C000002AABD1AA7805A93B88087130000A705C
:1078D0004B80FEF747FBA0E72845FF1FC8BF0011FC
:1078E0001D4B37B5050098420BD000290AD1FFF790
:1078F00077FF002805D11948FFF772FF002800D054
:10790000058037BD01291AD1FFF76AFF041EF8D0A0
:1079100001235B420380A378FF2BF2D0FE2B07D01C
:107920000023E0781422009329001E3300F032FB7C
:10793000A01C00F054FB01235B426380E1E70229B5
:10794000DFD1013901F0BEF80028DAD12800FFF7B5
:1079500047FF041EDFD1D4E7FEFF0000FFFF000059
:10796000022210B5074B52421A80074801325A8052
:107970009A80DA8000F07EFA044801F025F80020B1
:1079800010BDC046DC66FF1F05780011E1780011CC
:107990000388F7B50400002B02D102252800FEBDA4
:1079A00042680221137825485268FEF7A5FD002899
:1079B0002ED0234F01253A88002AEFD0802321883A
:1079C0005B0201259B1A9942E8DC0C2003F040FF82
:1079D000061E31D03B8822889C4600231800019562
:1079E00061469DB2491989B2AA421BD8002801D02C
:1079F00062443A8000233000082208C0210004F0CD
:107A0000C7F9104A1368002B13D100251660C5E78B
:107A10006268022113780C485268FEF76DFD002859
:107A2000C7D1BAE760681D0140194181013301984F
:107A3000D6E71A001B68E6E71325AFE736C000114A
:107A40002645FF1FD866FF1F34C00011014B187078
:107A50007047C0462845FF1F14230A0010B51A407E
:107A6000194204D00122102101F048F810BD4B0644
:107A7000F9D4012088434000F8E710B514008B06C4
:107A800004D50122102101F039F810BD08230A00A5
:107A90001A40194202D14BB2002B0FDA102101F02B
:107AA0002DF8002808D02300F9331B78002BECD0E8
:107AB000F8342378012BE8D10020E6E7032089077A
:107AC000FAD4E2E7F0B51F00184B85B01C680190AE
:107AD00002910392002C27D1200005B0F0BDA568CB
:107AE0003301ED186B89019A934211D3029A9342A4
:107AF0000ED8002F04D10A9B002B10D12C00EBE7ED
:107B00003B002978039A6868FEF7F6FC0028F2D15A
:107B10000136B6B2A388B342E1D82468DAE7A36895
:107B20000A9A5B891380E9E70026F3E7D866FF1F0E
:107B300037B50C000A8849880123914217D3002ADF
:107B400015D0651D23792A0002210A48FEF7D4FCCE
:107B5000102300280BD023796188208800242A0074
:107B60000094FFF7AFFF0A23A04200D023001800C3
:107B70003EBDC04636C0001113B50A0008884988CA
:107B8000012388420BD8002809D00024137905323C
:107B90000094FFF797FF0A23A04200D023001800AB
:107BA00016BD13B50A0008884988012388420BD8FE
:107BB000002809D00024137905320094FFF782FFD2
:107BC0000A23A04200D02300180016BDF0B58BB0E8
:107BD00003904A8808880E000123824255D300286A
:107BE00053D00023012704AC2370002271881300B6
:107BF0000092FFF767FF051E3ED02078002835D1A0
:107C00002B78022B18D167706A8983000130E31842
:107C100080005A8069680222201804F0B9F823789D
:107C20000133DBB22370042B19D93B006889013082
:107C300080B2002BD9D01FE0022363701223584377
:107C40006A89231804305A8069681022201804F0C9
:107C50009FF823780133DBB22370002BE5D10C4A67
:107C60006B899B185A425341DBB2DFE76378012BE3
:107C7000E4D12B78022BC7D022780A23002A04D023
:107C800021000398FEF798F9002318000BB0F0BD0F
:107C90000100FFFF0F4BF0B504001868002816D054
:107CA00083685D89A54207D88288AE18B44203DA9A
:107CB00012019A18934201D10068EFE71E005F8914
:107CC0001036A74204D1002900D00D801800F0BD65
:107CD0003300EFE7D866FF1F70B505000C00088879
:107CE0000021FFF7D7FF03000120002B04D0220062
:107CF0002800197AFFF7C1FE70BDF7B50C0000250A
:107D000001902300F6331B78AB4201D800200AE033
:107D10006B00E65A00213000E718FFF7BBFF002890
:107D200002D126800130FEBD017A0198FFF794FE52
:107D3000002802D03B882380F5E70135EDB2E0E76B
:107D400010B5040008880021FFF7A4FF03000120FC
:107D5000002B03D02000197AFFF77EFE10BD000033
:107D6000054B1B68002B01D1180004E09A6852896A
:107D70008242F6D198887047D866FF1FF0B50E276B
:107D8000002687B0039302ABFF183E8005001F4B0F
:107D900040891400984207D02B78013000976A6818
:107DA00080B2FFF78FFE060002212B7818486A6820
:107DB000FEF7A2FB00280FD06C892000FFF7D0FF50
:107DC000002802D0013C0419A4B2039B002B00D070
:107DD0001C80300007B0F0BD02212B780D486A6886
:107DE000FEF78AFB0028E7D102212B780A486A684F
:107DF000FEF782FB002807D0002EDED03B88A3428E
:107E0000DBD17489013CDFE76C89DEE7FFFF00000E
:107E100036C0001134C0001132C0001110B50C0082
:107E2000FFF7DEFC03000220002B0AD0002C00D05C
:107E300023609B781720FE2B03D00138FF2B00D145
:107E4000002010BD73B50D0001A904001600FFF756
:107E5000E5FF172805D0002E04D129002000FEF7E9
:107E600027F976BD01221021200000F047FE0028EE
:107E7000F3D0F6E7014B18607047C046E866FF1F75
:107E800037B56B469D1D010004000222280003F057
:107E9000AFFC2B88B02B0ED12379122B09D12300F4
:107EA000FF339B78012B06D10121608800F0E0F8B8
:107EB00001E01B2BF8D037BD10B5054B042118701D
:107EC00000F098F8FFF74CFDFEF770FB10BDC046C0
:107ED000EC66FF1F0020F0B50BB20F0087B08342A5
:107EE00034DA274B187803F08BFD051E2BD003786E
:107EF000A02B25D103AE3100FEF7E4F8041E0BD110
:107F0000B378DB0724D51F4B06341B68002B03D046
:107F10003100688898470400A868002801D003F061
:107F20000FFD002C08D1184A039B1340174A9342B7
:107F300006D0B3781B2B03D00121688800F098F895
:107F4000280003F065FD80200002784007B0F0BDF6
:107F50000F4B1B68002B10D0310068889847041E17
:107F6000DAD07378002BD7D1B27801A90A704B8090
:107F70000C716888FDF7F6FFCEE70624F1E7C046EE
:107F8000EC66FF1FE466FF1F00FFFF000001120008
:107F9000E866FF1FF7B50190822040000D00170032
:107FA0001E0003F015FC04001320002C12D0B02397
:107FB00020002370089BFC226770658026710830C2
:107FC000002B08D0190003F0E3FE2100019803F014
:107FD00047FD0020FEBD089903F012FEF5E710B53D
:107FE000041E06D00078FD2803D803F0C9FBFF2348
:107FF000237010BD0A1F93B210B504000220032B9A
:1080000005D882400020024BD1529B189C7010BDB5
:108010000C67FF1F0B8870B5043B04000D000220A5
:10802000032B0BD80121200000F04CFD030014208D
:10803000002B03D02900200000F0DEFB70BD000003
:1080400007B51300034A00920A00012100F02CFC3E
:108050000EBDC0467D82001107B501920322009239
:10806000024B0A00122100F049FC0EBDFB820011F8
:1080700007B56B4601AA11800449D88008780633F9
:10808000012802D1190003F033FC07BDED66FF1F84
:108090000C4B10B518700023FF210B4A138013817D
:1080A00093819380094A5380137051729381937224
:1080B000D174D3821375517703F08AFD00F0FCF977
:1080C00010BDC0461C67FF1F0C67FF1FEE66FF1F39
:1080D000F0B58DB06B46002003910C229B5E83426D
:1080E00000DBB0E05D4B187803F08AFC051E00D180
:1080F000A4E00378902B00D09DE006AF01004688F5
:10810000380000F013FA79680400002900D19CE0DF
:108110003B88052B6ED13B89032B1CD905AC200075
:1081200000F0A2F86288172A61D83989131D994294
:1081300031D17968237804310291D90738D5607834
:1081400000F08EF9071E06D0002303712378012B5F
:1081500008D0132B23D0A868002800D178E003F0C2
:10816000EFFB75E06288029909A800F0A6F802907A
:10817000380000F08BF909AA2378387A019200229E
:1081800031000092029A00F012F9380000F064F910
:10819000029B002BDFD0300000F080F9DBE7037892
:1081A000032BD8D16288029909A800F0D6F8DEE73F
:1081B000122B13D1029909A800F0B5F8021EEAD1DA
:1081C00027498B88002BC6D0887909A9237801918B
:1081D00061780091310000F0EAF8BCE7002302AAC0
:1081E00093833000617809AAFFF72AFFB3E71D4B9C
:1081F0000993F6E7042B02D09A1F012AABD8184A3C
:10820000043B9B00995A0029A5D0D21890783100E0
:108210003A0000F0AEF800289DD13B88042B03D033
:1082200001213000FFF724FF012C04D1A8680028A9
:1082300001D003F085FB280003F0EAFB8020039BBC
:108240000002434018000DB0F0BD012800D182E7C4
:1082500001213000FFF70CFFEDE7C0461C67FF1F50
:108260000C67FF1F010017000B7803704B784370F9
:10827000CB788A781B021343438070470A88030037
:1082800002700A88120A42700A88012A06D14A88B6
:1082900082704A88120AC27004207047022082420B
:1082A000FBD14A8804309A704A88120ADA708A88A8
:1082B0001A718A88120A5A71EFE710B5040001207A
:1082C00082420CD94B780A781B02134323808342E5
:1082D00006D1CB788A781B0213436380002010BD3F
:1082E000022BFBD1CB788A781B02134363804B7936
:1082F0000A791B021343A380F0E70B8803700B88F5
:108300001B0A43704B8883704B881B0AC3708B8891
:1083100003718B881B0A4371CB888371CB881B0A3E
:10832000C3710820704703000120082A14D14A783D
:108330000878120202431A80CA788878120202432F
:108340005A804A790879120202439A80CA79887958
:10835000120202430020DA80704710B504000120A9
:10836000022A05D100204B780A781B021343238090
:1083700010BDF8B5060010200F00150003F028FA14
:1083800004000120002C0ED0A0230C222900238001
:108390006780201D002D07D003F0FAFC210030007B
:1083A00003F05EFB0020F8BD03F02AFCF6E7F7B50A
:1083B0001E00009008AB142017001D78019103F0F7
:1083C00007FA041E12D0A2230370019B477043805A
:1083D000099B057146710C220830002B07D019004B
:1083E00003F0D6FC2100009803F03AFBF7BD099991
:1083F00003F006FCF6E737B5041E0FD04388002BC8
:108400000CD00025C1881323007A1722019500950E
:10841000FFF7CDFFFF2365806372257037BD000035
:1084200010B50C4904004A88002A09D08B89002B1A
:1084300005D00020CB8A0222834201D010BD012248
:1084400013000A20434300204032C854C818428019
:108450000472F3E7EE66FF1F00234380037070474A
:10846000094B00211A0010B55C88002C06D01C793D
:10847000844203D10A234B43D01810BD01310A3383
:108480000329F1D10020F8E7EE66FF1F10B50400C4
:10849000407A03F075F9FF23637210BD7047043012
:1084A00010B580B203F06CFB002803D004214942D0
:1084B00003F0EEFB10BD000070B50025104CA06865
:1084C0002580A581A580A84202D003F039FAA560D5
:1084D00000250C4C0C4B606D1D80230058331D7023
:1084E000A84202D003F02CFA6565002560680028D8
:1084F00001D003F025FA013508340A2DF6D170BDFC
:10850000B467FF1F5867FF1FA867FF1F70B5041EE1
:1085100009D1054D2880A881A880A868002802D02C
:1085200003F00EFAAC6070BDB467FF1FF0B54B8866
:1085300085B00193002343600A7905000F00022AE9
:1085400000D07BE0CA88032A17D98B685E78197837
:108550003602DC78D8790E4399781B7A24021B0204
:108560000C43034353495BBA0B80331D93421ED126
:10857000042C04D0631F022B0ED9012015E0019AB0
:108580004D4B1201D35A002B06D00198FFF7BEFFC6
:108590004A4A1369013313610421B8682E812C8083
:1085A000494203F075FB6860002005B0F0BD434D03
:1085B000042C06D0631F022B0FD9EB680133EB604C
:1085C000DBE7019A3C4B1201D35A002B05D00198EE
:1085D000FFF79CFF2B6901332B61374B300002936F
:1085E000019B029A1B010193002301998C468B5237
:1085F000130063449C8003939E81FFF750FF039B0D
:10860000041E986016D00421B868494203F040FB6C
:10861000FA880100043A200003F0BAFB0199029A9B
:10862000FB888A5A043B9B18029A8B522B680133B1
:108630002B60A2E7AB690133AB619EE71E4B02934F
:10864000019B1E01029BF35A002B2DD002998C191D
:10865000A068002828D0012A26D1FA889B189BB24E
:108660007352A189994217D39B1AC018B96803F0B5
:108670008FFB029BA289F35A934200D07DE7002230
:108680002B81A3882B80A3686B60029BF2520B4A5C
:1086900053680133536070E7084A9368013393606D
:1086A0000198FFF733FF68E7044A536901335361C8
:1086B000F6E7C0461E67FF1FB467FF1F2467FF1F52
:1086C00070B5051E15D10B4C0B4B18802300583389
:1086D0001870606D002802D003F032F9656525003E
:1086E00050356068002801D003F02AF90834AC4204
:1086F000F7D170BD5867FF1FA867FF1FF0B51700BF
:10870000A12285B0920001934243394B06001B68B9
:108710000C009B18D933FF331D78FDF741FF04305F
:10872000854204DD3000FDF73BFF0430C5B2BD4299
:1087300007D33A0000213000019B03F041F805B057
:10874000F0BD2900380003F043F92300C6B25033CE
:108750001E700393019B29006365380003F018FA2B
:10876000CBB20293002B02D0039B01361E70002671
:108770002300503303931B78B34204D8606D002864
:1087800031D10020DBE7029A2800002A04D0013B07
:108790001000B34200D02800F700E719387003F04A
:1087A0009FF8786000280ED03A78019903F0F0FA2B
:1087B000019A3B780136D3180E4A0193D369F6B279
:1087C0000133D361D4E7039B18706065A74205D1DC
:1087D000084A1320D36A0133D362B0E7606803F01C
:1087E000AFF80834F2E703F0ABF800236365C8E79D
:1087F0003409FF1F2467FF1FF7B50D000700042190
:10880000686803F045FA2B89040003702B891B0A62
:1088100043702B8883702B881B0AC3702E89022516
:108820000436F6B2FB2E15D81B4B9F4214D10C20F8
:1088300002F0CEFF1135011E0CD0902303708E3B49
:108840000371043B4380154B8460C680187803F0A5
:1088500007F900252800FEBD5C237B43104AD3188E
:108860000093583301931B78002B0FD10300320083
:1088700038000099FFF742FF019B05001B78002B91
:10888000E8D13800009903F013F9E3E7054A07251A
:10889000536A01335362DDE7FEFF00001C67FF1FD0
:1088A0005867FF1F2467FF1FF0B587B0009017209F
:1088B0000F0016000193FFF7F2FD1325041E19D0D7
:1088C0000C98031E02D00199201D9847030AE370FB
:1088D000052302AAA070043090812770009866706A
:1088E00003A993800494FFF787FF051E02D02000A0
:1088F00003F026F8280007B0F0BD0000F0B587B0FF
:108900001F000CAB1B780391059301210DAB0600F2
:108910001C78049200F0D6F81425002821D02000FD
:10892000FFF77EFD0135041E1BD01149059B0A7817
:1089300003700132D2B2131EC68001D101231A0086
:108940000B7022713000049B03990097FFF7ACFF76
:10895000051E09D1230021000648074A093302F009
:1089600067FF280007B0F0BD002363802370F8E79D
:108970002067FF1FF783001130750000F8B5050070
:108980000E00064C064F2368002B02D03100280051
:1089900098470434BC42F6D1F8BDC046C467FF1FF7
:1089A000D867FF1F0123064A5B42538000231371DF
:1089B0005362044A136053609360D360136170473D
:1089C000D867FF1FC467FF1F0200002310B50649C8
:1089D0009C000859002801D1625010BD0133052BBD
:1089E000F6D11320F9E7C046C467FF1F034A538836
:1089F000181A43425841404210407047D867FF1F41
:108A0000F0B585B002930AAB1F780CAB1B880090C1
:108A100008000E0001920393FFF7E8FF0500112004
:108A2000002D1BD10E48FFF7E1FF04001520002C9C
:108A300014D006220B99A771E01D03F0A9F9019B40
:108A400030002371029B29006371009B66802370B4
:108A5000039B6562E381FFF791FF280005B0F0BD3D
:108A6000FFFF000010B5FFF7C1FF04000220002C3B
:108A700012D060880121FFF781FF606A002801D0D1
:108A800002F0AEFF28220021200003F0B9F80123F4
:108A900000205B426380207110BD000030B5074AA2
:108AA000074C5588010013780020A54204D05B1ABA
:108AB00059424B415842104030BDC046D867FF1F55
:108AC000FFFF0000084A10B501230C00904208D0B7
:108AD000FFF78CFF031E04D0037923405A1E9341F5
:108AE000DBB2180010BDC046FEFF0000024B187933
:108AF000431E9841C0B27047D867FF1F70B504008D
:108B00000D001600FFF772FF002804D10D4B9C42A8
:108B100000D0143070BD416A03790520002907D0C8
:108B200012221A40102A02D10520002EF2D10F2065
:108B3000DB06EFD5897E0C20A94289414942494292
:108B40000840E7E7FEFF0000030010B5002800D151
:108B500010BD0348034A41889142F9D09847F7E78E
:108B6000D867FF1FFFFF0000002330B5C45CCD5C59
:108B70006C40D4540133102BF8D130BD0F230022A8
:108B800010B5C45C64002243CA54C25CD209013BE4
:108B9000F7D210BD0200010010B52032103102F0F2
:108BA00007FE10BDF0B58BB00390102005931700A1
:108BB000049102F04DFE0090102002F049FE009B4F
:108BC00013240190002B05D000280CD11324009809
:108BD00002F006FF019B002B02D0180002F000FFFC
:108BE00020000BB0F0BD102002F032FE0600102075
:108BF00002F02EFE13240500002E00D1AEE0002866
:108C000019D01022002102F0FBFF32002900039846
:108C100002F0CEFD041E0ED133787F2B51D83000E8
:108C20000099FFF7ABFF009B1B787F2B53D801996E
:108C30000098FFF7A3FF300002F0D2FE002D02D013
:108C4000280002F0CDFE002CC1D1102002F000FE61
:108C50000600102002F0FCFD0290002E7CD00028BF
:108C600078D03A000F3223000125121105D00F33BE
:108C70003B4015B25A4253411BB26A1E1201002BEF
:108C800033D0049BD2B298180099029AFFF76CFF78
:108C9000013D10220021300002F0B2FFADB2049F6E
:108CA0002D017D19AF4242D0002C33D0300002F0AC
:108CB00097FE029B002B00D189E7180002F090FE7E
:108CC00085E729003000FFF759FF28002549009A61
:108CD000FFF74AFFA7E729000098FFF74FFF28009A
:108CE0002049019AFFF740FFA5E70F210F400499A3
:108CF0008A18D9B28F4208D9D15C06A81954013319
:108D0000102BF6D1029A0199C0E7791A48424141E5
:108D1000C901F2E73900300006AAFFF725FF32004B
:108D2000039806A902F044FD10370400BAE7002CAE
:108D3000BCD13000029906AAFFF716FF320006A93F
:108D4000039802F035FD082204003100059803F075
:108D50001FF8ABE71324A9E71324AAE7002800D0E3
:108D60006EE733E73CC00011F0B58BB00F00160082
:108D70000225009000283FD0002A3DD00B1DDBB219
:108D80001800029302F064FD1135041E34D0FDF783
:108D900047FD05003A000099201D02F059FFEBB293
:108DA0000393E3702B0CDBB22F0A00936370FFB2C6
:108DB0002B0E2370A7700193FDF72CFD10220100EC
:108DC00006A802F045FF2100029A04AB06A8FFF7AF
:108DD000E9FE051E0DD1039B08223370009B04A9F8
:108DE000B370019B7770F370301D02F031FFFDF717
:108DF0001DFD200002F0F4FD28000BB0F0BDF0B521
:108E00008FB00D00149E039004920593002A03D1A5
:108E1000022420000FB0F0BD002EF9D00398FFF718
:108E2000E5FD1424071EF4D07278337812021A4339
:108E3000B3781B041343F27812061A43036A0192B3
:108E4000934201D30133E3D1002D03D03B790124B8
:108E50009B07DED50822002106A802F0D1FE059B63
:108E600013240433DBB21800029302F0F1FC051E58
:108E7000CFD0059A0499043002F0EAFE04223100B2
:108E8000280002F0E5FE3900102210310AA802F095
:108E9000DFFE2900029A06AB0AA8FFF783FE041E34
:108EA0000FD1082206A908A802F0D2FE0822311D1F
:108EB00008A802F0C5FC012807D101990398FDF725
:108EC000C9FC280002F08CFDA3E70124F9E70000AB
:108ED00070B51C4C05002368181E10D0002D14D14D
:108EE0001A78002A0CD1981C083202F051FF02F0C7
:108EF000EFFD0135002808D123681D70012070BDE9
:108F00000A331800082202F043FF2368002BF5D033
:108F1000122002F05DFC061E0DD0C12321680370F3
:108F2000457002311022023002F032FF2368310016
:108F3000587802F095FD206802F052FD002323606E
:108F4000DCE7C0460068FF1FF8B504002020FDF7ED
:108F500055FB0D4EA700BB590500002B0DD0002876
:108F60000BD0D878FF2809D108492A000C55F359AD
:108F700007480333611802F05BFCF8BD290002F0DA
:108F8000F7FB0028F0D1F8E71C68FF1F0468FF1FFB
:108F9000A1A1001170B5064D84006359002B05D0C6
:108FA000D87802F0EDFBFF226359DA7070BDC0463D
:108FB0001C68FF1F70B506008CB00C001500002166
:108FC0003022684602F01CFE31001022684602F092
:108FD0003FFE1D2021000322684402F039FE68464E
:108FE000FFF7D8FD2D21040003222800694402F078
:108FF0002FFE20000CB070BDF0B50700160097B032
:1090000001931CAB1D7830221EAB00910AA80021F1
:109010001C7802F0F5FD102239000AA802F018FEB3
:109020001022002102A802F0EBFD0722310002A865
:1090300002F00EFE072202AB9818631E9C410199B4
:1090400002F006FE02AB9C732B005A1E934102AA4B
:10905000D3730021102206A802F0D2FD06221D992A
:1090600007A802F0F5FD1A2002ABC01806221F99CE
:1090700002F0EEFD102200990EA802F0E9FD102288
:1090800002AB0EA908781C78013A6040D2B2087091
:1090900001330131002AF5D10AA8FFF77BFD102228
:1090A00012A904000EA802F073FE102206AB0EA94E
:1090B00008781D78013A6840D2B208700133013156
:1090C000002AF5D10AA8FFF765FD04431022209875
:1090D000E4B212A902F0BCFD200017B0F0BD70B5DB
:1090E0000E0014008CB00100102268461D0002F032
:1090F000AFFD3100082204A802F0AAFD21000822D9
:1091000006A802F0A5FD6846FFF744FD0400102202
:10911000280008A902F09CFD20000CB070BDF8B535
:1091200006000D0000243719AC4200D3F8BD02F050
:10913000F7FB030A3B70631CDBB201379D4203D986
:109140000234F054E4B2EEE71C00EDE773B506001C
:109150000C000225002819D0002917D0032101A8EE
:10916000FFF7DDFF6B469A793F231A400133134323
:109170006A463000937101A92200FFF71BFF051E0C
:1091800004D10322E01C01A902F002FE280076BDF2
:1091900003785807DA08C00FD20080009B071043FD
:1091A0009B0F1843C0B2704707230B40C908C90082
:1091B0000B4303707047000070B50400FFF7EAFE30
:1091C000134DA4006359002B21D0186A002801D048
:1091D00002F006FC2B59986E002801D002F000FC2A
:1091E0002B59D86E002801D002F0FAFB2B59186FCA
:1091F000002801D002F0F4FB2B59586F002801D051
:1092000002F0EEFB285902F0EBFB00232B5170BD5E
:109210001C68FF1F0E4B8000C35870B50C00002B5C
:109220000FD09D68002D0CD02B78201D0B706B7813
:109230004B70A97CFFF7B8FF2B7E23726B69E3604C
:1092400070BD10220021200002F0DAFCF8E7C046D1
:109250001C68FF1F014B18607047C0461868FF1F4D
:10926000074A03008000825810B5002A06D0D08833
:10927000984203D1012901D1FFF79EFF10BDC046DE
:109280001C68FF1FF0B5264E95B087000B93BB59A5
:109290000500099112200A92002B31D0D888FFF7DF
:1092A000A5FB04001420002C2AD0280010A9FFF7E9
:1092B000B1FFBB591E781D6A002E23D00895FDF71B
:1092C000EFFA07000020FDF7F1FA0790A379E61DF9
:1092D000069310AD0CA9089800F0E2FA0EA9280038
:1092E00000F0D7FA0B9B0A990493069B0998029306
:1092F000079B0396019300970EAB0CAAFFF77CFE29
:1093000015B0F0BDFDF7CCFA06903000FDF7CEFAAF
:10931000E31DA779079310AB06000893DAE7C04670
:109320001C68FF1F30B50C4C85002A59030085B01E
:109330000120002A0ED018006946FFF76BFF2B5959
:109340001A78D888054B002A00D1054B6A460721B8
:1093500000F0D9FB05B030BD1C68FF1F93980011C9
:10936000A198001130B5094C8500295985B010220B
:109370006846253102F00CFD2A591121044BD08892
:109380006A4600F0C0FB05B030BDC0461C68FF1F38
:109390003D99001130B5094C8500295985B010223E
:1093A0006846353102F0F4FC2A591121044BD0886B
:1093B0006A4600F0A8FB05B030BDC0461C68FF1F20
:1093C0007B990011F7B54D4F86001020F4590D0020
:1093D00002F03EFAF3592062186A132200286CD07A
:1093E000033A29009C6802F0D3FCF3591A780192E1
:1093F000002A58D11E6A227D317B944651400122B9
:10940000019F114201D167461740217D91433943A5
:109410002175377B4F40BC4660460027800701D44A
:109420004F081740012102208F40227D82433A439A
:109430002275377B5740BC4660460027400701D461
:1094400097080F400420227DBF0082433A432275D3
:10945000627D002794466046727B42400A4201D1F9
:1094600067460F400121627D8A433A436275777BEC
:109470005740BC4660460027800701D457080F407C
:109480000220627D7F00824317436775767B00224E
:109490007E40760701D4BA080A400426617D920016
:1094A000B1430A4362756A78002A08D06278002ABC
:1094B00005D005220533DA7700221000FEBD042214
:1094C0002979114205D1A17C114202D10533033A19
:1094D000F1E7019A21782C78002A02D10A002100B4
:1094E000140018220429E8D8042CE6D8052060438B
:1094F000034A05331218525CDDE7C0461C68FF1FA3
:109500004CC0001110B50A001121024B00F0FBFA0B
:1095100010BDC046D79900110B0030B587B001AD22
:109520002B806B4604001100981D082202F030FCCD
:109530002A000B212000024B00F0E5FA07B030BDF5
:10954000FF99001110B50A001121024B00F0DBFA5F
:1095500010BDC046539A001113B50B0011006A46A6
:1095600013706B4604000622581C02F011FC6A4678
:1095700008212000014B00F0C6FA13BD739A0011B8
:1095800010B50A001121024B00F0BDFA10BDC04613
:10959000C39A00117FB505000B4BAA00D4580800F0
:1095A000002C0FD0666F237FE28821780396266F08
:1095B0000296E66E0196A46E0094FDF709FC280061
:1095C000FFF7FAFD7FBDC0461C68FF1F10B51721CD
:1095D000FFF7E0FF10BD000070B50A000D00064B5C
:1095E0000221040000F08FFA060029782000FFF71E
:1095F000D1FF300070BDC046A399001170B586B090
:1096000000236A461370836804001D78681E0A28C8
:1096100059D801A902F064FA060633373B3F4347A5
:109620004B4F5300180000F042F9062312284BD08C
:1096300000281BD16088FFF7D9F90823002813D030
:109640004279002A47D1264B1A78072312070BD5F7
:10965000244B1A680723002A06D01668002E03D070
:10966000290001AAB04703006A4613706B461B78B5
:109670006088002B2AD1FFF767FC06B070BD180088
:1096800000F06CF9D4E7180000F087F9D0E7180073
:1096900000F093F9CCE7180000F0ADF9C8E7180026
:1096A00000F0C3F9C4E7180000F0F6F9C0E71800AD
:1096B00000F0F6F9BCE7180000F013FAB8E718005C
:1096C00000F013FAB4E707236A461370694660880E
:1096D000FFF782FFD1E70523012AC5D1024BB8E786
:1096E000A966FF1F1468FF1F1868FF1FF8B52C4FED
:1096F0008600F35904000D00002B40D0DA88824226
:109700003DD15A78062A33D11A78002A2ED001206A
:1097100099681A6A097D014206D0157B054203D07B
:1097200007225A700120F8BD0220014204D0157BA7
:10973000054201D00922F4E70420014204D0127B43
:10974000024201D00B22ECE7164B1B68002BE9D03C
:109750005B68002BE6D020009847BB5900215B785E
:10976000122BDFD12000FFF715FFDBE70E4BECE7F4
:10977000112A04D1002900D032252900F2E7002D5A
:1097800008D12000FFF732F9002803D01023027916
:109790001343037121002800FDF798FAC2E7C04681
:1097A0001C68FF1F1468FF1F1868FF1F70B50E4E5E
:1097B0008500AB590400002B13D01B78002B11D16E
:1097C0000A4B1B68002B04D05B68002B01D02000E3
:1097D000984773595B78122B03D100212000FFF7C3
:1097E000D9FE70BD024BECE71C68FF1F1868FF1F15
:1097F0001468FF1F094B8000C3581020002B0CD0A9
:109800001A6A002A09D09B68002B06D0127A1B7EA8
:10981000101C9A4200D9181CC0B270471C68FF1F68
:1098200070B503000D0014000220002A30D000297A
:109830002ED013700B78081D53704B789370FFF780
:10984000A7FCE070012002212B7A23716B7B03407F
:1098500063716A7B0A401343042263716E7B164076
:10986000334363716E7BF608F600334363712B7BE1
:109870000340A371287B014000200B43A371297B87
:109880000A401343A3712A7BD208D2001343A37169
:1098900070BD10B50A0001000120FFF7C1FF10BD27
:1098A00010B50A0001000220FFF7BAFF10BD70B525
:1098B00006000C000220002E30D000292ED0737834
:1098C000201D0B70B3784B70F178FFF76DFC01220F
:1098D0003579257271794B10080013409340104080
:1098E0000343881010408000C9080343C9000B439C
:1098F0006373B1794B100800134093401040034349
:10990000881002409200C9081343C9000B4321206C
:109910002373FCF773FE854201D2122070BD222012
:10992000257AFCF76BFE8542F7D823781820042BA4
:10993000F4D86378012BF1D80020EFE7030010B5CD
:109940000220002909D0002B07D00322481C0A70EE
:1099500019000D3202F01CFA002010BD0300022293
:10996000080010B5002B06D0002904D00E32591C77
:1099700002F00EFA0022100010BD030010B5022004
:10998000002909D0002B07D00422481C0A701900B6
:109990000C3202F0FDF9002010BD10B5FFF7DEFF1C
:1099A00010BD03000220002906D0002B04D00522A0
:1099B00000200A701B784B70704703000220002BB8
:1099C00008D0002906D05B7800200B70013B082BE3
:1099D00000D918307047030010B50220002909D0C3
:1099E000002B07D00622481C0A7019000A3202F028
:1099F000CFF9002010BD10B5FFF7B0FF10BD020079
:109A00000B00022010B500290ED0002A0CD007212F
:109A10001970118859701188090A99701118082253
:109A2000D81C02F0B5F9002010BD03000A00022086
:109A300010B5002B0CD000290AD09978587809026B
:109A400001431180901CD91C082202F0A1F90020CA
:109A500010BD030010B50220002909D0002B07D04B
:109A60000822481C0A701900921802F091F900208F
:109A700010BD02000B00022010B500290BD0002AF7
:109A800009D009211970117818185970511C062233
:109A900002F07EF9002010BD10B5FFF75FFF10BD8A
:109AA00002000B00022010B5002A09D0002907D0BF
:109AB0005178197011180622581C02F069F900201B
:109AC00010BD030010B50220002909D0002B07D0DB
:109AD0000A22481C0A701900063202F059F90020C7
:109AE00010BD10B5FFF73AFF10BD02000B000220B9
:109AF00010B5002A06D0002904D018005178FFF7CD
:109B000053FB002010BDF0B585B017001E006A465B
:109B100006230500080091819380FEF7C0FC132402
:109B2000011E02900CD03800B047041E05D1280059
:109B300001A9FEF76FFA041E02D0029801F000FF9F
:109B40002800FFF701FA200005B0F0BDF0B50400D1
:109B50008BB0019115000021102202A802F050F8EC
:109B6000334EA700B85900283CD0C388A34239D14E
:109B70000378002B36D14278062A18D10200010062
:109B8000553235310C3006ABFFF7A9FA002829D140
:109B90002000FFF72FFE020006A902A802F0F8F845
:109BA000200002A901F0B4FE01200BB0F0BD816ECF
:109BB000002917D00B8A112A28D19D420ED1019875
:109BC0001231093A01F03CFE012807D1BB592000AF
:109BD0009D6EFFF70FFE29000200DEE73221200014
:109BE000FFF7D8FC2000FEF701FF061E1BD0416ADC
:109BF000002918D00B8AAB4215D1082201981231E6
:109C000001F01EFE01280ED1716A0AE09D42E9D1E1
:109C100008220198123101F013FE0128E2D1BB594C
:109C2000996E8A7EB9E7200002F002F8BCE7C046D0
:109C30001C68FF1FF0B56B4D87007E5985B03378E7
:109C400002900393002B00D087E0B368346A01933D
:109C50007078062817D101221B7D134202D0217B88
:109C6000114218D10222134202D0217B114251D15C
:109C70000422134203D0237B134200D08BE0019BCC
:109C80005A7DEB5991E007380428F8D801F028FFF5
:109C9000032E42678300B36E002B03D11C2001F01A
:109CA000D7FDB066EB599C6E002C1CD01022002111
:109CB000200001F0A5FF0298FFF79CFD01002000A5
:109CC000FFF72DFA01F02CFE20822000082112302F
:109CD000FFF725FA0298FFF78DFDA076EB592100DA
:109CE000D888FFF70FFC0822EB591CE0B36E002B5D
:109CF00005D01A00198AF0881232FFF70DFC0222F3
:109D0000019B197DEB5911423DD0207B10423AD086
:109D1000073208E0F488FCF7DBFD01002000FFF7C4
:109D200011FC0A22EB595A70029B9C002A59537865
:109D3000073B042B11D8D088FEF758FE00284ED0E0
:109D4000C3895A08D2182849029B0298CB542B5930
:109D500041180433254801F06BFD05B0F0BDFCF758
:109D60009FFD03000120834201D100200393EB59A2
:109D7000DE88FCF79BFD039902003000FFF7ECFB47
:109D8000019AEB59117D042211420CD0217B114222
:109D900009D00B22C7E7F688FCF73CFD0100300034
:109DA000FFF7EEFB6BE7019A527D01210A4204D0D6
:109DB000607B084201D00C22B5E702210A4204D0A0
:109DC000607B084201D00E22ADE704210A4204D094
:109DD000627B0A4201D01022A5E71222A3E7FA22F1
:109DE0005200B0E71C68FF1F2068FF1FABA10011E5
:109DF00010B5064B1A780423100018401A4200D000
:109E00000348FFF727FA002010BDC046A966FF1FD0
:109E10002C45FF1F70B50400FFF7D4FA051E43D18F
:109E20002000FFF77FFA234EA400A0598268937C9C
:109E3000DB0708D50321036A1B790B40012B02D1F4
:109E4000017F0B430377431DD97F8B1E022B0DD857
:109E5000022900D00121C088FCF790FF042133596A
:109E60001A7F59700A431A77280070BD01290CD156
:109E700002231022437000210C3001F0C1FE305942
:109E800010213530FFF74BF9EEE70529ECD102231D
:109E9000D118437010220C3001F07AFF042332599C
:109EA000117F0B431377EAE708251828DCD1053D1D
:109EB000DAE7C0461C68FF1FF0B58BB005914388F8
:109EC0007E4F9E00F45915000493002C15D10129F2
:109ED00002D000200BB0F0BD101D57781678FFF7A8
:109EE00057F9EB68320002932B7A049901930090A2
:109EF0003B002000FCF70CFFEBE7E388049A934259
:109F000001D00820E6E72378012B00D1D4E0059B9F
:109F1000581E092800D9CFE001F0E2FD05CE0A293C
:109F2000CC506C859AB229000498FFF773FFD1E7F3
:109F3000200029001022453001F02AFFB9594B7842
:109F4000042B02D1013B4B70C3E70B000A00253301
:109F500035320C310498FFF795F90498FFF702FAAF
:109F60000522431E9841BB59C0005A70B2E7200039
:109F700029001022553001F00BFF049B4F4C9D002F
:109F8000295904980A0006AB55320C31FFF77AF9CB
:109F900029591022453106A801F052FC012808D1A8
:109FA0000498FFF7F7F90590002804D106222B59F1
:109FB0005A7005988EE708230593FAE763780C2B0F
:109FC0007AD1E36E002B03D11C2001F041FCE06646
:109FD000BB59D86E00286FD01022290001F0D8FE9E
:109FE000BB590498DC6EFFF705FC0D22A076BB5927
:109FF0005A706EE7E06E00285ED063780D2B5BD15F
:10A000002B8808220382A91C123001F0C1FEBB5923
:10A010009A68517D0222114226D0186A407B104274
:10A0200022D00C32E4E763780E2B45D1236F002B4E
:10A0300003D1162001F00CFC2067BB59186F0028D3
:10A0400003D01022290001F0A3FE0F22BB59CFE755
:10A0500063780F2B30D1206F0622691C103001F07D
:10A0600097FEBB599A68517D0422114203D0196AA8
:10A07000497B1142D5D100210498FFF78BFA28E7DC
:10A08000636F002B0DD0BB59586F0028F3D01022FE
:10A09000290001F07DFE0122BB5952425B6F1A611B
:10A0A000E9E7142001F0D4FBBB5960675B6F002B1C
:10A0B000E9D126E72978DFE707200BE71C68FF1FB7
:10A0C00010B5064C207001F0ABFD06212078FDF79D
:10A0D00091FF0348FEF778FC10BDC0462F68FF1FB4
:10A0E0006192001100200BB270B50D00834216DAA8
:10A0F000264B187801F084FC041E0DD00378922BB7
:10A100000ED0A02B37D0224B1878FF283AD0210050
:10A1100001F0A6FC002835D180200002684070BD07
:10A1200043780E2B0BD03E2BEDD18378052B12D02C
:10A13000082BE8D181798088FFF7D8FA08E0154B21
:10A1400082889A42DFD183681878591CFEF7C0FED6
:10A15000002817D1D7E7104B1B785B0712D50F4BA0
:10A160001B68002B0ED09B68002B0BD0C289811D71
:10A1700080889847ECE7FFF741FAA068002801D0F3
:10A1800001F0DEFB200001F043FCC5E72F68FF1F54
:10A190002545FF1F18200000A966FF1F1868FF1F34
:10A1A00010B50078FFF712FA10BD10B50078FFF770
:10A1B000FDFA10BD0C234343084A10B59B185A689A
:10A1C000002A03D0012901D1904710BD9B68002BC4
:10A1D000FBD00029F9D19847F7E7C0464C68FF1F2C
:10A1E00010B5162813D801238340094A946B1C43E9
:10A1F0009463506B98435063D46B200098430129BB
:10A2000001D120001843D063116B0B43136310BDC1
:10A2100000800040F0B500240127154B85B0DA6BB3
:10A22000144E03921A6C0192DA64019BE3403B42A4
:10A2300017D0039DE5403D400295E5B20299280004
:10A24000FFF7B8FF316A736A002908D03900002B84
:10A2500001D0029979402800FFF7C2FF01E0002BEE
:10A26000F9D101340C36172CDFD105B0F0BDC04652
:10A27000008000403068FF1F10B50124020020005C
:10A28000162A08D8054B5968D140214204D01868D5
:10A29000D0400123184010BD186DF9E70080004040
:10A2A000162807D80122064B8240002903D0D9681E
:10A2B0000A43DA607047D9689143D960FAE7C0462B
:10A2C0000038004030B5162818D8032444430F4BFB
:10A2D000E25C1B199C785D7801232D1B0135AB4096
:10A2E000013BA340A140DB430C00122807D80849DA
:10A2F00092005218116819402143116030BD054A7F
:10A3000011680B4023431360F8E7C04693C0001167
:10A3100008F0004014F00040C21F70B5D4B206230C
:10A32000092C0BD80125084C9540002908D00021A4
:10A33000FFF7C8FF23682B4323600023180070BD7C
:10A340002368AB43F8E7C04600380040F0B5162854
:10A3500026D8214B1B185B78022B21D103244443C0
:10A360001E4A1F4EA35C12199478012215008540E5
:10A37000B76B013CE4B23D43A240B563194C1228CF
:10A3800015D89B0000290CD117495B1899680A431E
:10A390009A600123205C154A834011680B431360C7
:10A3A000F0BD11495B18996891439960F1E70E4B34
:10A3B00000290DD159690A435A61225C1328E8D05B
:10A3C0000123203A93400A49086803430B60E7E7FA
:10A3D000596991435961F0E73068FF1F93C000113C
:10A3E00000800040D8C0001100F00040A0F0004004
:10A3F000A4F00040F8B500241B4E1C4D1C4B1B5D07
:10A40000012B1FD1184A9269E2401A420BD0012257
:10A41000AA5693402200143AD2B2022A09D815490A
:10A420004A6913434B6101340C360235172CE5D1D0
:10A43000F8BD0022AA560F499200521891680B43AA
:10A440009360F0E7022BEED1E7B23800FFF714FF7C
:10A4500001235840C1B23800FFF778FF3800FFF7FA
:10A460000BFF7077DFE7C0463068FF1F65C0001143
:10A470003168FF1F00F00040012202388240054B86
:10A48000002903D059690A435A61704759699143B9
:10A490005961FAE70038004070B504000D0005204E
:10A4A000162C1AD800212000FFF7FAFEA31E012B5C
:10A4B00003D801212000FFF7DFFF00212000FFF774
:10A4C0002BFF01220A49A2400A4B4868012D05D101
:10A4D00002431B194A605D70002070BD90434860C4
:10A4E00002211C196170996991439961F4E7C04692
:10A4F000008000403068FF1F10B516280AD80122DE
:10A50000074B8240002906D019680A431A600121CE
:10A51000FFF7C2FF10BD196891431960F7E7C04605
:10A520000080004070B505000520162D17D80C23BB
:10A5300000246B430A4A21009B181C70094B280019
:10A540005B195C70FFF7A8FF0123AB4020000649B0
:10A550000A681A430A6005490A689A430A6070BD8E
:10A560004C68FF1F3068FF1F34800040308000407F
:10A5700070B504000E00FF2813D003250540FFF737
:10A58000D1FF084AA3089B009B183F22ED00AA4078
:10A59000AE40196820009143314319600121FFF753
:10A5A0007FFE70BD18380040F8B505000520162D57
:10A5B00025D80C246C43124BE4186368002B03D19C
:10A5C000A3680D30002B1AD0022201270D4B002169
:10A5D0005B195A7028002770FFF75EFF63681E1E24
:10A5E00008D0A3683E00002B04D02800FFF744FEEB
:10A5F0004640F6B228003100FFF7F2FD0020F8BD1A
:10A600004C68FF1F3068FF1FF7B5C420FF222B4B9B
:10A6100080001958002491437F3A0A431A5080223F
:10A62000274F5202274E1A60274B1D5D002D21D067
:10A63000A31E012B03D80121E0B2FFF71DFF012D5E
:10A6400018D11F4B9B69E3402B4213D0E3B2180093
:10A650000193FFF711FE01000198FFF74DFFE3B2F0
:10A66000143B022B1DD801217156184A8D405369A5
:10A67000AB4353613B7F002B0DD0E5B22800FFF7C1
:10A6800093FF2800FFF7F8FD7B7F0100834202D093
:10A690002800FFF78FFD01340C370236172CC3D189
:10A6A000F7BD012100237156F3568D40074A9B00E8
:10A6B0009B189A68AA439A60DCE7C04600E100E074
:10A6C0003068FF1F65C000113168FF1F00F00040B7
:10A6D00010B504000520162C0CD801212000FFF72E
:10A6E000DBFE0123044A002011194B70A34091693D
:10A6F0000B43936110BDC0463068FF1F70B50E005C
:10A7000015000400FFF70EFF0C236343094A2000E5
:10A710009B189D605E60FFF747FFF021064B074ADC
:10A720008900051E5A5002D02000FFF7FBFE2800CA
:10A7300070BDC0464C68FF1F0000FF1F15A200112E
:10A7400070B5134D07202C78002C1FD198222100C2
:10A750005200280001F0F4FA0123C420FF222B70DC
:10A760000C4B80001C635C630B4B1C605C600B4BF0
:10A77000195891437F3A0A431A50802252021A60B4
:10A780000D20074A074901F0FBFA200070BDC046C2
:10A790003068FF1F00800040A0F0004000E100E0B2
:10A7A00009A60011F5A30011030010B50620072B20
:10A7B00009D8054A137001F05BF8D7210020034B3C
:10A7C000034A89005A5010BD5445FF1F0000FF1F67
:10A7D000151BFF1F70B51D0002240C2910D8094A53
:10A7E000CA40D2070CD5FBF715FF041E08D1059A05
:10A7F00004992800FBF72AFFFCF798FDFFF7F8FA09
:10A80000200070BD1210000030B50D7802232C001E
:10A810009C43184201D02B431C0008252300AB4366
:10A82000284201D02B00234320241D00A5432042B1
:10A8300001D01C4325002A230D70184204D0117842
:10A840001E3B0B43137030BD0028FCD10C21137844
:10A850008B43F7E7F8B51D0006AB1B88140007AA69
:10A860000E000B201778002B27D10A78022A49D135
:10A870004A68507811780002244A08438018042856
:10A8800040D801F02DF903121D1B2300F06801F0E0
:10A89000BFF9021CC0B2B84200D93A1CD2B22000A3
:10A8A000F1682A8001F074FA06E00222F3681B883E
:10A8B0002A8023701B0A63700020F8BD0622EEE791
:10A8C00001232B80F3681B782370F5E7F368002BD6
:10A8D00016D008222A801A8822701A88120A6270FA
:10A8E0005A88A2705A88120AE2709A8822719A884D
:10A8F000120A6271DA88A271DB881B0AE371DBE756
:10A900002B80D9E701202B80D7E7C04600D6FFFF78
:10A91000F7B516000A781D0008AB1F880C0001234C
:10A92000022A18D14A685078117800022B4A08434D
:10A93000801803280FD801F0D3F802254439E068C5
:10A9400001F066F9C0B20723B84204D37B19019322
:10A95000152B02DD0D231800FEBDE0682A00310032
:10A96000C01901F015FA6B4600209B88E268D054AC
:10A970001B4B1B68834203D01B68834200D098475F
:10A980000023E8E70B23002FE5D1022DE2D17378F5
:10A9900032781B021343E2681380114B1B68002BB3
:10A9A000EED01B68002BEBD00120E8E70B23002F33
:10A9B000D1D1062DCED12A003100E06801F0E8F9AE
:10A9C000DEE70B23002FC6D1012DC3D132787533BA
:10A9D000012AC0D8E3681A70D2E7C04600D6FFFF4C
:10A9E0003C6AFF1F70B50C001500072837D801F02E
:10A9F00077F8041436361B36242E182015290BD868
:10AA0000184E16220021300001F0FAF82200290029
:10AA1000300001F0BDF9002070BD18200229FBD1E3
:10AA20001288114B1A80F6E718200829F4D10A0081
:10AA30000E48290000F0DCFEEDE718200129EBD1DB
:10AA40000B4B10780B49DA69FFF7DEFEE3E71820BD
:10AA50000129E1D1064B10780749DA6BF4E70220AF
:10AA6000DAE7C046246AFF1FD245FF1FC845FF1F13
:10AA70005845FF1F8045FF1FA045FF1F030010B56D
:10AA80000020DB0704D50721024A034800F08CF8B8
:10AA900010BDC046F0C000115845FF1F054A030015
:10AAA0001068002803D082889A4201D180687047DC
:10AAB0000068F6E7406CFF1F0A88030008009A420E
:10AAC00004D08A8804309A4200D0002070470000E9
:10AAD000F8B5F82200230D4F0D4E7968050042436A
:10AAE0003370994200D07B600A4C0021200001F0B5
:10AAF00087F800231A007C60AB4202D1002033703B
:10AB0000F8BD01332280DBB2F834F5E7406DFF1F5A
:10AB10003C6DFF1F446CFF1F73B56B460190060030
:10AB2000684615001980FCF733FF041E11D1002D73
:10AB30000FD07689002E11D00C2000F089FE00285D
:10AB40000ED0084A0460136886808560002B02D10D
:10AB50001060200076BD1A001B68F7E70224F8E7B2
:10AB60001324F6E7406CFF1F012100220A4B10B5A9
:10AB700049420A4C198099809A719A70084B20704A
:10AB8000012019805A60FFF7A3FF2078FCF75EFFD1
:10AB90000448FDF719FF10BD446AFF1F486DFF1FF1
:10ABA000406DFF1F55AC0011022310B5002802D0E4
:10ABB000FFF7B2FF0300180010BD0000030010B53E
:10ABC0000020DB0704D50421024A0348FFF7A4FF55
:10ABD00010BDC04604C10011D845FF1FF0B50E26B8
:10ABE00087B003930CAB1F8802ABF6180500080072
:10ABF00031000292FDF74EF804000120002C0FD026
:10AC00003088FFF74BFF03000E20002B08D05E6852
:10AC1000002E05D021002800039B029A0097B04720
:10AC200007B0F0BD0A4B10B5984207D101220023AE
:10AC300052420A808B708A808B7110BDFFF73CFFF7
:10AC40000028FAD001235B42038000238370F4E7DD
:10AC5000FFFF0000F8B5050001290AD1134E0024BA
:10AC60003388F827AB4219D028001149FFF7DAFFE3
:10AC700006E0022904D10139FDF724FF0028EDD0B8
:10AC8000F8BD3B0063437268D018D35A002B09D03B
:10AC90003A00002100F0B4FF0134E4B2054B1B7808
:10ACA000A342EED801235B423380DDE7406DFF1FF6
:10ACB000446AFF1F3C6DFF1F10B5FFF7FDFE030048
:10ACC0000020834200D0987810BD0000F0B589B014
:10ACD0001C000EAB80CB03901E8810AB1B78049237
:10ACE00002930B7A0D00DB0616D42B780593022B0A
:10ACF00024D00498FFF7D2FE002812D003689C46A7
:10AD0000002B0ED0029B2200019329003B006446D9
:10AD100003980096A04705E00498FFF7BFFE0028BF
:10AD200002D10E2009B0F0BD8368002BF9D00A22B1
:10AD30002900039898470028D7D0F3E76B68587824
:10AD40001A786B4B000210439842D2D8043B9842C9
:10AD500010D2684B984242D015D8674BC0180128D2
:10AD6000C7D80B20002EDDD1EB681A7859683A80DD
:10AD7000200028E0614BC018032800D979E000F0DA
:10AD8000AFFE846A789E5E4B9842B2D10B20002EB3
:10AD9000C8D101233B80EB6831001B7823706889A0
:10ADA000013080B2FCF776FF3A88031E0ED001789E
:10ADB00002328A183A80428962704289120AA2706D
:10ADC00059680278E01C00F0E3FF06E004323A80A4
:10ADD00031000422601C00F013FF0020A2E70B20CA
:10ADE000002E9FD1EB6807A91E8804233B80330AFD
:10ADF000300026706370FCF74DFF051E28D004ABB1
:10AE00009A890E2304A95B183E49C668FCF7B6FF71
:10AE100000280BD12B783C486A680599FBF76CFB3E
:10AE2000002803D1012304AA5B42D3813278022A8D
:10AE300006D17168201D00F0ABFF3B8802333B80D8
:10AE40000E2304AA9B181B88A3701B0AE370C4E797
:10AE500004ABDE81F4E70B20002E00D062E7E96846
:10AE60000398FFF729FF02233B802070000A6070DF
:10AE7000B3E70B20002E00D054E70222EB681B88BA
:10AE80003A8023701B0A6370A7E7E86800F0C0FEF1
:10AE9000C2B203000720B24200D243E70DD00299AC
:10AEA000DBB27118994202DB921BD3B20293029B70
:10AEB000E9681A003B8089195AE70023F6E70B205E
:10AEC000002E00D02EE70722EB683A801A78227015
:10AED0005A7862705A88A2705A88120AE2701A79F7
:10AEE0002271DA886271DB881B0AA37175E7C0469C
:10AEF000042900000228000000D8FFFFFFD6FFFF52
:10AF000003280000FFFF000034C00011F0B58DB031
:10AF10006B460020089120229B5E83423DDAA64BBF
:10AF2000187800F06DFD071E32D00378B02B2CD1BD
:10AF30000079023816281FD800F0F2FD17001E0015
:10AF40001E001E0031001E0096001E001D011E0086
:10AF500052011E0073011E00CD011E0050021E0092
:10AF60001E001E008E021E00E302944B94491B88B3
:10AF700078880B80FBF700F83800FCF781FF914BD5
:10AF80001B68002B01D038009847380000F040FDC6
:10AF90008020089B0002434018000DB0F0BDF6224F
:10AFA0000021874800F02CFE0BAA3B7B7989388969
:10AFB00000923A000D32FCF785FD0400804B1B78AF
:10AFC000002C3FD146E0804B788805937F4B4100B1
:10AFD000CB5A0BAE073BDBB23288029300230193BE
:10AFE0007B4B210006930093059BFFF76FFE744D8A
:10AFF000002810D1069B3A8A1B889A420BD1380050
:10B000000599123000F01CFC002804D02B786289CE
:10B010009B00EB185A80162306A81B1832882000C4
:10B020007989FCF7ABFE2B7804009A00AA185188A6
:10B030000029C3D00133DBB22B70002807D006A94A
:10B04000C98A9180634A12889A42BCD802E00121E1
:10B0500049429180002B04D059497888FAF7C0FF03
:10B060008AE73E890A2479E000253E89574B0693FA
:10B070007B88069A5B009B5A033B9D4202DB002DB6
:10B08000F0D05BE0162206A812183B7B798900926B
:10B090003A0030000D32FCF715FD0590002858D01D
:10B0A0004689017A7888FCF7D7FC041E44D1464BC8
:10B0B00078880793069B4100C95A454B0439C9B2A9
:10B0C00006AAD28A06930291019400930599079BE0
:10B0D000FFF7FCFD041E2FD1069B39491A88931CEB
:10B0E000002D26D14B807988384B4900CB5A511915
:10B0F000033B8B4220DD059B31485B8941190B7175
:10B10000A91C0135C9B2EDB2059145191B0A2B7175
:10B11000059B2D490433181800F03AFE2C4B059A74
:10B120001B88D318DDB22C4B9E4205D00136B6B237
:10B130009CE749889942D6D0002D0CD0204C28009D
:10B14000618800F0F5FA207021007888FAF758FF3E
:10B1500012E7059CF0E7002C00D183E77B78142BE5
:10B1600000D109E716493B794E800B700C71788845
:10B17000FAF7F8FE00E7162406ABE4182100388938
:10B18000FCF788FD011E00D1B7E1788822880F4CBA
:10B1900045002C5B0A4D013CE4B2029400240F4BA5
:10B1A00001940095FFF792FD041E00D014E12900E0
:10B1B0007888FAF735FFDFE6486DFF1FC444FF1FAC
:10B1C0004C6AFF1F406AFF1F466BFF1F7C66FF1F14
:10B1D0003C6CFF1FC244FF1FFFFF00004E6AFF1FB1
:10B1E000162406ABE41821003889FCF753FD011E34
:10B1F00000D182E178882288AE4C45002C5BAE4DB0
:10B20000013CE4B202947C89AC4B01940095FFF7B9
:10B210005DFD041E00D0DFE029007888FAF70AFF00
:10B22000AAE60025A44B1D803B00FE331B78A24AF2
:10B2300078880792AB4208D99E4B128806930699EC
:10B2400043005B5A013B9A4203DB0799FAF7FCFE85
:10B2500092E616246B00FB18059306ABE418059BD9
:10B2600021001889FCF716FD011E03D1059B01245E
:10B270001E8973E77888924B2288069C09934300C5
:10B280001B5B904E013BDBB20293002300960193BF
:10B29000099BFFF71BFD041E02D0059B1E895DE77D
:10B2A0007B88069A5B009B5A079A1088328812188E
:10B2B000934202DC1B1A013B33807F4C0230328800
:10B2C0000999001900F064FD2388328801359B1824
:10B2D0002380EDB2A8E70BAA3B7B798938890092DD
:10B2E0003A000D32FCF7EEFB00250590059B002B84
:10B2F00004D10A24002D00D16EE060E0059B78881F
:10B30000197AFCF7A9FB0100041E63D1694C6C4B50
:10B31000788806940993069B4400E45A694B063CDE
:10B32000E4B20BAE32880793029401910093059921
:10B33000099BFFF7CBFC041E4CD1079B5E491B8881
:10B340001A1D002D30D14A80059B5B4C5A89631928
:10B350001A716B1C9BB2E318120A1A71162306A805
:10B3600032881B1879890598FCF708FDFF21AA1C73
:10B370002E1D03350B00059092B2B6B2ADB2002877
:10B3800003D006ABDB8AD9B21B0AA218651911716A
:10B390002B714C4D301D2A884949201800F0F8FCCB
:10B3A0002B88F618B5B2A1E74988914207D17A886F
:10B3B00006995200525AEB18053A9A42C4DC3E4CA8
:10B3C0002800618800F004FB207021007888FAF7DB
:10B3D00045FED1E5002DF2D13E89BFE6162606AB2B
:10B3E000F61831003889FCF755FC3D000400FF35A4
:10B3F00000282DD0037A9B060CD400227B89398942
:10B40000788800923A000C32FFF7E8FB041E10D057
:10B410003E8915E03088FFF741FB00281AD0836889
:10B42000002B17D02100122278889847041EE4D000
:10B43000EEE7AB78002B02D17888FAF71FFE0026E2
:10B44000AB78002B00D097E5002C00D194E585E681
:10B450000124DDE70E24DBE7162506ABED182900F5
:10B460003889FCF717FC041E47D0037A9B0611D4D9
:10B47000154A7B881188994203D01448814207D12C
:10B480001380134BF8261D780023D9B2A94221D38B
:10B490000924A1E72888FFF701FB00282FD0836843
:10B4A000002B2CD02100122278889847041EDFD070
:10B4B00092E7C0467C66FF1F4C6AFF1F4E6AFF1F63
:10B4C000466BFF1F3C6CFF1F406DFF1FFFFF00001E
:10B4D0003C6DFF1F31005943546801336018615AB5
:10B4E0000029D2D13C0008342100F82200F050FCA1
:10B4F00021007888FAF7CAFD3EE501246CE70E24A6
:10B500006AE71D4B1A887B889A4231D07888FAF70F
:10B51000C7FD31E5F823059851684343CD18C95A52
:10B5200000291FD03B7A012B0BD16C88AB8878881F
:10B53000AA1D0094FFF752FB041E02D000233B72A9
:10B540002E88F8220021280000F05AFB00232B80CF
:10B55000059B0133DBB20593084B05991B78064A1E
:10B560008B42D7D801235B421380002CCED0F5E567
:10B57000002634000596EFE7406DFF1F3C6DFF1F6E
:10B5800070B504000E001500FFF796FA031E08D1EF
:10B5900031000548FFF790FA03001120002B02D07C
:10B5A0001C8000209D7070BDFFFF0000F8B50B4FA0
:10B5B00006003B780D001400FF2B0ED00A2000F08F
:10B5C00007F9011E09D0B1230380002346800371CF
:10B5D000C5800481387800F043FAF8BD1946FF1F92
:10B5E000F7B50F0008A90600088809A90B240988E7
:10B5F000002821D10234022B1ED1557813782D0258
:10B600001D432B008B4301937334002B14D1FB6833
:10B61000300019000093FFF74FFB019C85420BD0CF
:10B620002A0030000099FFF7ABFF041E04D12A0066
:10B6300030007989FFF7BAFF2000FEBDF0B50E7823
:10B6400085B003900AA805880120022E0DD14C6810
:10B650002778647824023C43054FBC4205D1039807
:10B66000DBB201960095FFF7BBFF05B0F0BDC04609
:10B670000229000010B504000C4800F051F80C48F5
:10B68000A16B00F04DF80B48E16B00F049F80A4857
:10B69000216C00F045F8094B0948196800F040F8A2
:10B6A000084B1B68002B00D09847FEE7E6BE001150
:10B6B000FCBE00110BBF00111ABF001104ED00E029
:10B6C00029BF00114C6DFF1F002307B501A801938E
:10B6D000FFF7D0FF044A0548002110B5121A00F008
:10B6E0008FFAF8F767F9FEE7506DFF1F1C46FF1F42
:10B6F00001B40248844601BC604700BF8552010086
:10B7000001B40248844601BC604700BFC521000067
:10B7100001B40248844601BC604700BF3136FF1FB8
:10B7200001B40248844601BC604700BFE53A01000D
:10B7300001B40248844601BC604700BF350E0000DA
:10B7400001B40248844601BC604700BFF30E00000C
:10B7500001B40248844601BC604700BFDD660100B9
:10B7600001B40248844601BC604700BF291C0000A8
:10B7700001B40248844601BC604700BF5147010044
:10B7800001B40248844601BC604700BF1147010074
:10B7900001B40248844601BC604700BF6932FF1F04
:10B7A00001B40248844601BC604700BFC9A900003B
:10B7B00001B40248844601BC604700BFE548000070
:10B7C00001B40248844601BC604700BF5118FF1F06
:10B7D00001B40248844601BC604700BF1D4D010012
:10B7E00001B40248844601BC604700BF8132FF1F9C
:10B7F00001B40248844601BC604700BF810E0000CE
:10B8000001B40248844601BC604700BF9130FF1F6D
:10B8100001B40248844601BC604700BFA54F010047
:10B8200001B40248844601BC604700BF5D170000B8
:10B8300001B40248844601BC604700BFA94601002C
:10B8400001B40248844601BC604700BFCD4C0100F2
:10B8500001B40248844601BC604700BF3D4B010073
:10B8600001B40248844601BC604700BFDD30FF1FC1
:10B8700001B40248844601BC604700BF151BFF1F8E
:10B8800001B40248844601BC604700BFB14E0000CD
:10B8900001B40248844601BC604700BFB537FF1FB2
:10B8A00001B40248844601BC604700BF3D18000057
:10B8B00001B40248844601BC604700BF093AFF1F3B
:10B8C00001B40248844601BC604700BF4135FF1FF8
:10B8D00001B40248844601BC604700BFD13CFF1F51
:10B8E00001B40248844601BC604700BF017F0000EC
:10B8F00001B40248844601BC604700BFE117000064
:10B9000001B40248844601BC604700BFE134FF1F18
:10B9100001B40248844601BC604700BF311B0000EF
:10B9200001B40248844601BC604700BF29510100B0
:10B9300001B40248844601BC604700BF3939FF1F8B
:10B9400001B40248844601BC604700BFD9490100E8
:10B9500001B40248844601BC604700BFD53BFF1FCD
:10B9600001B40248844601BC604700BFADAE000090
:10B9700001B40248844601BC604700BF5522000064
:10B9800001B40248844601BC604700BF8538FF1FF0
:10B9900001B40248844601BC604700BFED4A010083
:10B9A00001B40248844601BC604700BF156B01002A
:10B9B00001B40248844601BC604700BFD1A5000025
:10B9C00001B40248844601BC604700BFEDA50000F9
:10B9D00001B40248844601BC604700BF090E000064
:10B9E00001B40248844601BC604700BF014C01001D
:10B9F00001B40248844601BC604700BFC95C010035
:10BA000001B40248844601BC604700BFF54E010006
:10BA100001B40248844601BC604700BF434D0100A9
:10BA200001B40248844601BC604700BFC51D000048
:10BA300001B40248844601BC604700BFC132FF1F09
:10BA400001B40248844601BC604700BF413AFF1F71
:10BA500001B40248844601BC604700BFB54C0100F8
:10BA600001B40248844601BC604700BF594F010041
:10BA700001B40248844601BC604700BFB3520100D4
:10BA800001B40248844601BC604700BF350E000087
:10BA900001B40248844601BC604700BFF539FF1F6E
:10BAA00001B40248844601BC604700BFC53F0000A6
:10BAB00001B40248844601BC604700BF7D18FF1FE7
:10BAC00001B40248844601BC604700BFC94A010076
:10BAD00001B40248844601BC604700BFD91B000086
:10BAE00001B40248844601BC604700BFE53CFF1F2B
:10BAF00001B40248844601BC604700BF691F0000D2
:10BB000001B40248844601BC604700BFC13AFF1F30
:10BB100001B40248844601BC604700BF9DA90000F3
:10BB200001B40248844601BC604700BFF93CFF1FD6
:10BB300001B40248844601BC604700BF595201006D
:10BB400001B40248844601BC604700BF813AFF1F30
:10BB500001B40248844601BC604700BF4550000064
:10BB600001B40248844601BC604700BFA134FF1FF6
:10BB700001B40248844601BC604700BF9137FF1FF3
:10BB800001B40248844601BC604700BFE9280000B8
:10BB900001B40248844601BC604700BF090E0000A2
:10BBA00001B40248844601BC604700BF2146010041
:10BBB00001B40248844601BC604700BF5125000023
:10BBC00001B40248844601BC604700BF8D120000EA
:10BBD00001B40248844601BC604700BF79180000E8
:10BBE00001B40248844601BC604700BF456B0100B8
:10BBF00001B40248844601BC604700BF851F0000B5
:10BC000001B40248844601BC604700BF154D0100E5
:10BC100001B40248844601BC604700BFDD52010008
:10BC200001B40248844601BC604700BFC926000039
:10BC300001B40248844601BC604700BF091B0000F4
:10BC400001B40248844601BC604700BF2D3BFF1F82
:10BC500001B40248844601BC604700BF4551010061
:10BC600001B40248844601BC604700BF6571010011
:10BC700001B40248844601BC604700BF8B520100FA
:10BC800001B40248844601BC604700BF252600007D
:10BC900001B40248844601BC604700BF5549010019
:10BCA00001B40248844601BC604700BF055E000045
:10BCB00001B40248844601BC604700BF056A000029
:10BCC00001B40248844601BC604700BF35550000FE
:10BCD00001B40248844601BC604700BF2124000033
:10BCE00001B40248844601BC604700BF1D4B0100FF
:10BCF00001B40248844601BC604700BFF94C010012
:10BD000001B40248844601BC604700BF6DBC00001E
:10BD100001B40248844601BC604700BF01890000AD
:10BD200001B40248844601BC604700BF0124000002
:10BD300001B40248844601BC604700BF4D1F0000AB
:10BD400001B40248844601BC604700BFB70E000042
:10BD500001B40248844601BC604700BFA93BFF1FF5
:10BD600001B40248844601BC604700BFC56D0100B4
:10BD700001B40248844601BC604700BF0D52010077
:10BD800001B40248844601BC604700BF0933FF1F6D
:10BD900001B40248844601BC604700BFE94C010081
:10BDA00001B40248844601BC604700BF75A9000089
:10BDB0000002010302020303040305020602070254
:10BDC000080209030A030B030C020D020E030F0302
:10BDD000100311031303140315001600913D001105
:10BDE000C53D00110000000002000000F2BD00117E
:10BDF000192A0F180A000000F1590000FD24000064
:10BE000041460100D1800011E5A0001139750011F3
:10BE1000D57E0011395300110DAF0011C54F00112F
:10BE2000D93F001109410011000000001616000062
:10BE3000020000003CBE0011F4FFF3FFD2FC000042
:10BE4000D541001100000000000000005475796128
:10BE50000042312E3000303030310067697468752F
:10BE6000622E636F6D2F70767678005448303500FF
:10BE70000200000084BE0011292A282A272A262A27
:10BE8000252A242A0A180000E2040000710200009A
:10BE900078EC0000744000001027000060F0000003
:10BEA00006640000204E00000000000001000000B9
:10BEB0001F501D00023CB4000001150010000000DE
:10BEC000A10200003031323334353637383941423F
:10BED00043444546005048592B36325858504C552B
:10BEE0005330353034005B48617264206661756C94
:10BEF000742068616E646C65725D0A004C5220208B
:10BF0000203D203078253038780A0050432020200A
:10BF10003D203078253038780A0050535220203D9B
:10BF2000203078253038780A0049435352203D208C
:10BF30003078253038780A003D57001191570011AC
:10BF4000000000000200000050BF00116F2A6E2A9E
:10BF50001A18EAC8BC80F0FC60FFFFFFFFFFFFFF7C
:10BF6000FFFFF303B59747D6F613F7D777E6F0A7A9
:10BF7000F474000001A00000000000006410B71D70
:10BF8000C8206E3BAC30D9269041DC76F4516B6B07
:10BF90005861B24D3C7105502083B8ED44930FF0C9
:10BFA000E8A3D6D68CB361CBB0C2649BD4D2D3867F
:10BFB00078E20AA01CF2BDBDFB349B5F80000080CC
:10BFC00000100000000000003B610011C577001167
:10BFD0005F610011CD7B0011E3610011A37B0011B3
:10BFE00059620011797B0011AB620011417D001193
:10BFF00013630011417D001145630011FB7C0011AA
:10C0000059620011317B0011D1620011D97C0011FD
:10C010000000000000000000B7630011D97C00118F
:10C0200019640011DD770011052A042A012A002A6B
:10C030000229032801280028011800180000000028
:10C040000000000000000000000000870101020164
:10C0500002010102010203030401030101010101C4
:10C060000303020103000D000E0010001100130075
:10C070001401070108010A010B011C011D02040241
:10C0800005020702080219021A021C021D0301031D
:10C09000020317000201000504000807000B0A0054
:10C0A0001716001D1C010201010504010E0D0111EE
:10C0B00010011413011716011A19020201020B0ACA
:10C0C000020E0D02111002141302171603050403C9
:10C0D0000807030B0A030E0D0001020307090A0BF0
:10C0E0000E0F101112141718191A1B1F20212200ED
:10C0F00055A8001111A90011000000000200000065
:10C100003AC00011000000003DB600110000000020
:08C110000200000038C000111C
:020000041FFFDC
:1000000000000000ED3E0011F8BD0011F4BD00112C
:100010002863FF1F00000000000000000000000037
:1000200000000000000000000000000000000000D0
:1000300000000000000000000000000000000000C0
:1000400000000000000000000000000000000000B0
:1000500000000000000000000000000000000000A0
:100060000000000000000000000000000000000090
:100070000000000000000000000000000000000080
:100080000000000000000000000000000000000070
:100090000000000000000000000000000000000060
:1000A0000000000000000000000000000000000050
:1000B0000000000000000000000000000000000040
:1000C0000000000000000000000000000000000030
:1000D0000000000000000000000000000000000020
:1000E0000000000000000000000000000000000010
:1000F0000000000000000000000000000000000000
:1001000000000000000000000000000000000000EF
:1001100000000000000000000000000000000000DF
:1001200000000000000000000000000000000000CF
:1001300000000000000000000000000000000000BF
:1001400000000000000000000000000000000000AF
:10015000000000000000000000000000000000009F
:10016000000000000000000000000000000000008F
:10017000000000000000000000000000000000007F
:10018000000000000000000000000000000000006F
:100190000535FF1F5533FF1FC16601000000000039
:1001A000000000000000000000000000000000004F
:1001B000000000000000000000000000000000003F
:1001C000000000000000000000000000000000002F
:1001D000000000000000000000000000000000001F
:1001E000000000000000000000000000000000000F
:1001F00000000000000000000000000000000000FF
:1002000000000000000000000000000000000000EE
:1002100000000000000000000000000000000000DE
:1002200000000000000000000000000000000000CE
:1002300000000000000000000000000000000000BE
:1002400000000000000000000000000000000000AE
:10025000000000000000000000000000000000009E
:10026000000000000000000000000000000000008E
:10027000000000000000000000000000000000007E
:10028000000000000000000000000000000000006E
:10029000000000000000000000000000000000005E
:1002A000000000000000000000000000000000004E
:1002B000000000000000000000000000000000003E
:1002C000000000000000000000000000000000002E
:1002D000000000000000000000000000000000001E
:1002E000000000000000000000000000000000000E
:1002F00000000000000000000000000000000000FE
:1003000000000000000000000000000000000000ED
:1003100000000000000000000000000000000000DD
:1003200000000000000000000000000000000000CD
:1003300000000000000000000000000000000000BD
:1003400000000000000000000000000000000000AD
:10035000000000000000000000000000000000009D
:10036000000000000000000000000000000000008D
:10037000C9B60011000000000000000000000000ED
:10038000000000000000000000000000000000006D
:10039000000000000000000000000000000000005D
:1003A000000000000000000000000000951AFF1F80
:1003B000000000000000000000000000000000003D
:1003C000000000000000000000000000000000002D
:1003D000000000000000000000000000000000001D
:1003E000000000000000000000000000000000000D
:1003F00000000000000000000000000000000000FD
:081838005071FF1F4118FF1F52
:10184000024981F3088802F013FB00005071FF1F6A
:1018500010B502F05DFB072804D0122808D002283A
:1018600008D010BD044A0420136B01331363F8E75A
:101870000220F6E71420F4E72467FF1FF8B50700FD
:101880000C0026002500503630785135002804D150
:101890000300287058342370F8BD2978CA00481E08
:1018A0008141A3183800A25C5B68C9B2FFF7D0FF82
:1018B00000280DD12B78DA00A218013350602B706C
:1018C0003378044A013B3370136A01331362D8E75B
:1018D0000123DFE72467FF1F5C234343074910B55B
:1018E000C9180B0058331B78012B05D1FFF7C6FF31
:1018F000034A936A0133936210BDC0465867FF1FC5
:101900002467FF1F10B502F013FA064A01211300E5
:1019100010CB4942D967044B136002F071FC2000E0
:1019200010BDC04600E100E01000100010B504003A
:1019300002F0FEF9024B1C6002F062FC10BDC046D2
:1019400000E100E010B5040002F0F2F94021094A7C
:10195000200013688B43136002F052FA01F0B4FDCB
:101960000022054B01201A60044B04321A6002F079
:101970004FFCFEE71CF00040C4F00040C0F0004007
:10198000431E5A425341A022F0B5D2015B4213409C
:10199000154D164A40019B182A18127E8BB00191F2
:1019A000002A1BD01A000832D46F0022E6B206AF1C
:1019B000E4B294420EDC2818C369002B08D00199C8
:1019C00002AA117106AA049202AA167303A89847E4
:1019D0000BB0F0BD1978B9540132EAE71A7D1A78D4
:1019E00006AB01261A70E6E7E469FF1F00400040DD
:1019F000F0B5254B04004001C25C85B0002A2BD015
:101A00001A18117E002927D0917E002924D011793F
:101A1000022921D11689D788D168F51BADB22A1CBD
:101A2000102D00D9102292B2BE4217D118180123EE
:101A300003710023C269C38003819A4206D06846BD
:101A4000032103730171029301A890470820002C21
:101A500000D0192001F034FC05B0F0BD013C654216
:101A60006C41A0256442ED012C40084D1B186419FF
:101A7000074D0633013A92B2AA42EDD01888461CAF
:101A80001E80085C2070F5E7E469FF1F00400040FD
:101A9000FFFF00000F220E4B10B59868104002386F
:101AA0000A280BD802F01EF90D0A0B0A0A110A0ABD
:101AB0000A0A060002210020FFF762FF10BD012183
:101AC000F9E70020FFF794FFF8E7DB6FF6E7C04681
:101AD000004000400F220E4B10B5986810400238AD
:101AE0000A280BD802F0FEF80E0A0B0A0A120A0A9C
:101AF0000A0A060002210120FFF742FF10BD012162
:101B00000800F9E70120FFF773FFF7E7DB6FF5E760
:101B10000090004013B5334C2378072B3DD8324B4F
:101B20001A78324B002A39D18022196852020A43AE
:101B30001A60252001F084FF20232D4A11680B43F1
:101B4000802113606B460422C905086807331042E0
:101B500028D080210422C905C86810422ED08021D7
:101B60002020C905CA688243CA6014221A701A78F4
:101B7000002A2FD18021C905C86820320243CA60DB
:101B800014221A701A78002A28D11A4B1A7D22784A
:101B90005A601D221A705932DA6013BD1A6816494C
:101BA0000A40C5E7086802430A6014221A701A78CE
:101BB000002ACED01A78013AD2B2F7E7C8680243B9
:101BC000CA6014221A7019784A1ED2B21A700029FB
:101BD000F9D1C4E71A78013AD2B2C7E71A78013AC4
:101BE000D2B2CEE75445FF1F1C46FF1F3CF0004019
:101BF0004C45FF1F00200040FFFFFEFF564B70B515
:101C00001B68012B03D1554A936D0133936502F094
:101C10000FFA534B534A1860534B544C1A6001232C
:101C2000534A1360534A13602378002B06D00622D0
:101C30005149524802F00CF900232370504A514B8D
:101C400010681B78C1B2002B0ED14F4CC0B2237864
:101C50005BB2002B4FDB237824785BB264B21B04A9
:101C600024021B191B1813600B1C50294ED950233A
:101C7000464A47491078DBB2FF2202284BD1086858
:101C8000444C454D267890432A78964254D9227880
:101C900024782E78023B5D10A31B6B435201D31AAC
:101CA00010335B111843086002F0A2FA031F012BE6
:101CB00045D83A4B1B78002B06D0394B1B78002BAC
:101CC00002D0002002F03CFAA122364B9200997813
:101CD000354B4A431B689B18832292009B181B7844
:101CE000033B012B03D8AF20400002F051F8012242
:101CF0002E4BDA8270BD237824785BB264B2FF3356
:101D0000FF341B0424021B190138ABE7CAB2022AB4
:101D1000AED20223ACE70868254C264D26789043C6
:101D20002A78964208D9227824782D78023B5B10D5
:101D3000641B63435201B2E72378DBB2B2E70228A7
:101D4000D5D11D4B1B78013B022B03D91B4B1B78B4
:101D5000022BCCD16C20C8E79809FF1FFC0FFF1F96
:101D60005C66FF1FFF3F0000141003406066FF1F0A
:101D70000C10034000100340D50BFF1F7211FF1F12
:101D8000B40003408C09FF1F680AFF1F490AFF1FA8
:101D900094000340460AFF1F470AFF1FF908FF1F70
:101DA0002209FF1F300DFF1F3409FF1FBC0BFF1F4F
:101DB000440AFF1F450AFF1F1C09FF1F2309FF1FBD
:101DC00010B502F00DF90022014B1A8010BDC0467B
:101DD0005866FF1F10B502F0EBF8A121054A8900F3
:101DE0009478054A61431268044B5218528C1A8049
:101DF00010BDC046300DFF1F3409FF1F5866FF1F7E
:101E000010B50D4B0D4A9978A1239B004B431268E6
:101E1000D218531DD97F0A4B1B88994209D2441C02
:101E200007D0C82805D0D2695B1A5A43054B5343E3
:101E3000C01802F05DF910BD300DFF1F3409FF1FFF
:101E40005866FF1F7102000070B5244D2B68002BEF
:101E500028D002F0E5F82B68D8402B680400002B4E
:101E600027D002F085F92B68D8401D4B1D4A997880
:101E7000A1239B004B431268D118D25C91239B0095
:101E8000002A20D0CA580132CA50174B17491B6884
:101E90000868834214D3D23B181A012A1AD0144B73
:101EA000186070BD02F0BCF8124B196802F0B8F966
:101EB000D3E702F05DF90F4B196802F0B1F9D4E7EE
:101EC0000D495B18E8E7CA500C4B1B68DB68E41847
:101ED000201AE4E7F530FF30E1E7C0461C08FF1F99
:101EE000300DFF1F3409FF1F9C09FF1F5C66FF1F99
:101EF000A009FF1F1808FF1F2DFF3F006466FF1F8A
:101F000070B504000D00282916D10300A433C2883F
:101F10001B889B1A0B4A9BB293420DD906006A3666
:101F200005223100653002F04BF9002804D1310060
:101F3000200002F0ADF870BD2900200002F038F951
:101F4000F9E7C046FE7F0000F8B50400012001F06B
:101F50006FFF02F04DF8174A174910600968030037
:101F60001648174E01601748776805680020AF4291
:101F700001D27068281A144D091928601348C162EB
:101F8000A421446A49032143416211490978002987
:101F900005D010490978022902D10F3B1360F8BD22
:101FA000012901D1083BF9E7032901D1053BF5E7F8
:101FB000033BF3E7E408FF1F28F00040340AFF1F4B
:101FC00028100040180AFF1F1C0AFF1F00F00040E5
:101FD0001C09FF1F4A0AFF1F70B580241025E40565
:101FE000A3682B43A36001F0EBFFA368AB43A3609E
:101FF00070BD0000F7B5160080221C001023D2052A
:102000000191916805000B43936000225A4BD73031
:102010001A6001F09DFF9D232A002F009B00EB58C2
:10202000CA3201210092FC37002B01D00021009A16
:10203000386801F07DFF2900009BCB311A784F4BA7
:10204000D3351A604B780A781B0213438A7812043E
:102050001A43CB781B061343494A1BBA13604B79CA
:102060000A791B0213438A7912041A43CB7931008F
:102070001B061343434A1BBA13606B782A781B0272
:102080001343AA7812041A43EB781B0613433E4A03
:102090001BBA1360019A330213433C4A13603C4B52
:1020A00022001B1B9C4603293DDCB3089A00130049
:1020B0005142B21A032A46D1354AE018511A8278A1
:1020C0004078120400020243E05C043302430A60D9
:1020D0000022FF2B4BDDF0222E4B12011A600F2243
:1020E0002D4B1A602D4A1368002BFCD00023224A86
:1020F00027491360091B321D0B191B68043A180A83
:1021000023706070180C1B0EA070E3700434002A5A
:10211000F2DC802210213B68D20501333B609368DA
:102120008B439360F7BD6346D578981893782D0656
:102130001B042B43157804392B43557804322D02A8
:102140002B430360AFE7022A0AD1114AE05C511A1F
:10215000E2185278120202430A6004339BB2B7E7D6
:10216000012AB5D10A4A521AE15C1160F5E7084923
:1021700059180A600433ACE7000004403C000440F6
:102180003800044034000440300004400C00044097
:102190000001044004000440100004401400044006
:1021A000F7B5150080221C001023D205009191681C
:1021B00007000B4393600023654AD730136001F09A
:1021C000C7FE9D233E009B00F9583B00CA363200F3
:1021D000FC33002900D07FE0586801F0A9FE3900E7
:1021E00032785C4BCB311A604B780A781B02134370
:1021F0008A78AC4612041A43CB78281D1B06134379
:10220000554A1BBA13604B790A791B0213438A792A
:1022100012041A43CB791B061343504A1BBA1360AE
:102220004B7A0A7A1B0213438A7A12041A43CB7A36
:1022300021001B0613434A4A1BBA1360009A2B0263
:102240001343484A13602200474B1B1B0093009B1B
:10225000CE785B1801938B7836061B0433430E78D7
:10226000043833434E78043136023343019E3360E1
:102270000328ECDC0321A808431C9B0029408000B4
:1022800003292BD13849E5185E18A9786D78E35CED
:1022900009042D022943194331600300083300214A
:1022A000FF2B2DDD314B324919600F21314B196065
:1022B000012327490B60304B19680029FCD0062107
:1022C0001B680B40042B20D080220020D20593688D
:1022D0000A318B439360FEBD01217DE7022908D1BD
:1022E00021495D18E1184978E35C09021943296026
:1022F000D3E70129D3D11C495918E35C0B60CCE723
:102300001948181801600433CAE7002310490B600C
:102310006346002B0CDC3B00FC335A681021013271
:102320005A608022D205936801208B439360D2E7E4
:10233000009B9B181B68190A13705170190C1B0E17
:10234000D37004235B4291709C440432E0E7C046A2
:10235000000004403C0004403800044034000440C5
:10236000300004400C00044000010440040004401C
:10237000080F0000100004401400044070B5061E51
:1023800019D00222614B9B799343012B13D1604BEF
:102390001A78FF2A0FD15A78FF2A0CD19A78FF2A8F
:1023A00009D1DA78FF2A06D11A79FF2A03D15B799D
:1023B000FF2B00D1A7E0574B0C201A78012A08D038
:1023C0000022554D1A702B781A00093A042A01D8B8
:1023D000212070BD5A1F012AFAD94C4CA07B042839
:1023E00000D990E0A279032A00D98CE0821E012A4C
:1023F00003D862881F2A00D885E0002E61D0012E04
:1024000000D080E0A288012AE2D0002B0AD1013856
:10241000032803D801F066FC151D19151F202E7026
:1024200001F0D6FE2B785A1E032A16D800253B4B06
:102430001D602823237501F01BFEA8422ED0A58025
:10244000C6E7022320202B70EAE7042322202B700A
:10245000E6E7032321202B70E2E7073B012BB7D8E7
:102460002F4B1B68DB6A9B06B2D52E4B1A78002ACD
:10247000AED1A27B911E012901D9002AA8D1022246
:1024800080211A702823284D89012878237501F0AE
:10249000CFFE80212878890101F05AFC0123A38016
:1024A000224B1B78002B0AD0FA228021204B92006D
:1024B0001B8809025A431C4B187801F0F9FC0020D4
:1024C00087E701F035FC2B78A680073B012B06D966
:1024D00018482E7001F014FE1E2001F079FE114BF9
:1024E000114C1A78002A06D0802100222078890118
:1024F0001A7001F09DFE01F083FE80212078090210
:1025000001F096FEDBE7122063E7C046A60BFF1F33
:102510006B09FF1F1A09FF1F1C09FF1F4809FF1F36
:102520006466FF1F2309FF1F1B09FF1F2109FF1FEF
:102530002C09FF1F0010004010B5002901D001F048
:102540008FFC10BDF7B5604B01919978A1239B00DA
:102550004B435E4A060014681022E418D6235B0041
:10256000E0583623FF33E35C00279343222B41D10D
:10257000574B0F3A1A600760012501F0D1FB019B10
:102580001880E8235B00E35C002B01D0B34258DDE8
:102590000023504FFB70AD33FF33E3581A68002A15
:1025A00003D09B88DB439B071DD03823FF33E35CBC
:1025B000002B18D09B235B00E35C002B13D1D1339D
:1025C000FF33E35CB3420EDAA4235B00E15AE01868
:1025D000090A023101F0DCFD23000122FE33013E35
:1025E00001351A87FA70E8235B00E35C002B2AD0E0
:1025F000A8B2FEBD03683D00002BBED08188043028
:10260000090A023101F0C4FDD6235B00E3581F60C4
:10261000B2E72300B133BA00FF33985801378188FD
:102620000430090A023101F0B3FDE8235B00E35CEA
:10263000BB42EEDCE822F61AED1800235200A35448
:10264000A6E70027F1E7200001F0C2FB00281FD019
:10265000002E1DDD7319882647190193B60020004E
:1026600001F016FC5A30800020184068013581883E
:102670000430090A023101F08BFD200001F098FBC3
:10268000A3590133A351BD4202D0019B9D42E6D123
:10269000114BE35C002BABD095239B00E35C002B3C
:1026A000A6D00E4BE15A0029A2D00D4AA35C994254
:1026B00002D90133A3549BE700231A212000A3541D
:1026C00001F026FB94E7C046300DFF1F3409FF1FC1
:1026D00000140340E010FF1F5A02000072020000C5
:1026E0005E020000F8B51D4B1D4F1A78002A10D16C
:1026F000BA7B002A02D101321A7003E0032AFAD011
:10270000022AF8D001F0B4FC00220120154B1A7007
:10271000F8BD154B154D1C68154B9E7801232B7089
:102720002878C0B200F0DEFCBB7B002B0BD101F09F
:102730006FFCA1239B007343E41883239B00E418E0
:1027400023782B70E4E7032B02D101F081FCF0E742
:102750000020022BDCD101F093FBEAE71C09FF1FEC
:10276000A60BFF1F2309FF1F3409FF1F490AFF1F84
:10277000300DFF1FF0B587B00EAD2F780FAD2D785F
:102780000593AC46634614000E4D0CAA12782E78C1
:1027900003930D9B009201932200059B029701F089
:1027A00097FC2E70012C01D0042C08D18022064900
:1027B0008B889343054A1278D20113438B8007B06C
:1027C000F0BDC0461C09FF1F6C11FF1F7809FF1FD9
:1027D0000B001B3B70B504003020E02B0DD813001C
:1027E000E025493BFF3B9BB2ED00AB4205D8034BD4
:1027F000200019825A8201F0E3FA70BD8410FF1F95
:1028000010B501F015FC054B00205B68052B04D9C1
:10281000034A5268D20200D4980810BD001000404C
:10282000FCE100E070B501F083FA0D4B1B68FC334E
:10283000DC691D6AFFF7E4FF6419844204D2094B86
:1028400001241B68002B07D004220024064B1A70B9
:10285000064A93690133936101F0D2FC200070BDF8
:102860006466FF1F9809FF1F2309FF1FFC0FFF1F4E
:1028700070B50C4D2B68FC335C6A01F059FAFFF718
:10288000BFFF2B680025FC339B6AE318834204D208
:10289000054B1B68AB4200D1051B01F0B1FC2800C1
:1028A00070BDC0466466FF1F9809FF1FD722044B06
:1028B00092009B5810B5002B00D0984710BDC04621
:1028C0000000FF1FF0B587B001F096F9FFF7EEFFAB
:1028D000CA4BCB4C04931B78022B45D1C94B1B68C8
:1028E000186A01F0A5FAC84BC84A1A60C84BC94A11
:1028F0001A60A022C84B52001A60049B187801F09D
:10290000BFFBC649C64801F08BFAC649C64801F06C
:1029100087FA1022C54BFF201A60802252031A60EA
:10292000802292031A60802212041A6001F008FCCF
:10293000012001F025FCFA20400001F0C1FB5820E5
:1029400001F026FABA4801F0C3FA012001F018FAA2
:10295000072001F07DFC2268B64B1A4084235B00FF
:102960001343236007B0F0BD01F0FAF9B24E0290B4
:10297000322001F05DFA33681B0629D43C2001F0B7
:1029800057FA0F2001F054FA9C4B1B78012B00D111
:102990001EE180223368A94D134200D0A7E02B68C6
:1029A000032013432B6001F043FA01F0D9F9029B95
:1029B0000299C31A5A1E814200D81A00A04B1A600D
:1029C000904B19681E2353439E4A9B18CB618AE79C
:1029D00001F0C6F980239C4ADB02116803900B4387
:1029E00013602268934B994F1A40282313432360A6
:1029F000032001F01DFA03203D6801F019FA3B683D
:102A00000320DB03DB0B009301F012FA3B68ED03BC
:102A1000DB03ED0BDB0B8E4A0193AB18C22B30D8D6
:102A2000009B9B18C22B2CD8019B9B18C22B28D82B
:102A3000009B2A009D4200D21A00009B9D4200D9B3
:102A40001D00019B934200D21300019A954200D9C8
:102A500015005B1B122B14D80C22336814209343EF
:102A6000336033687B4A1340336001F0E1F9082199
:102A70003B682268DB038A432260774ADB0B1360E2
:102A80007FE7032001F0D4F93B68DB03DB0B059300
:102A900001F066F9039B0399C21A531E814200D8C4
:102AA00013006E4A93421BD9FF23356869492D0AEA
:102AB0001D4032686B1C1B060A401B0C134333601D
:102AC0000C23326800209A43083B1343336001F023
:102AD000B7FB6348634BA840984206DCFEF732FF21
:102AE000019B009D0093059B95E75F48F6E7002357
:102AF0005E4F554A3B6080231168DB020B43136035
:102B000080222B68032013432B6001F091F93B686E
:102B1000052601333B6080232A685B0213432B6048
:102B20002268444B03201A40514B1343236001F0A9
:102B30007FF90821454B1A682368D2038B43236031
:102B4000454B023900931B68D20B4B439A420CD879
:102B50009B1A3B2B0BD8236846490B4023602B68FC
:102B60000B402B60444B1A601FE7D31AF1E7013E7C
:102B7000F6B2002ED4D123683E4A134023602B685E
:102B800013402B603B68042B07D9BFF34F8F3B4B9F
:102B90003B4ADA60BFF34F8FFEE780222B680320A9
:102BA00093432B6001F044F92268224B03201A4022
:102BB00028231343236001F03BF9244B009A1B6840
:102BC000DB03DB0B1360082223689343236097E742
:102BD00007222C4D2B681340012B02D1002001F05D
:102BE0004FFAAB68284A02201340AB6001F020F98D
:102BF0008023AA685B001343AB60D6E64A0AFF1F36
:102C00005CF000406466FF1F000003400180063D49
:102C1000BC00034034080000A4000340710200001F
:102C200014100040FFFF3F002810004000E100E0CA
:102C30003075000000FEFEFFC4F0004044F000408C
:102C40004C66FF1F7206000040F0004064F0004038
:102C500091FCFFFFFF00FFFF5466FF1FE30C000025
:102C6000E88000005F361E0060361E00B844FF1F7B
:102C700028000100FFFFFEFF5066FF1F00ED00E08F
:102C80000400FA053CF00040FFFEFFFF694E336888
:102C900088331B6883F3088801F09AF900F014FC6C
:102CA000654B664A1B68934207D0002001F0C8FAC2
:102CB0000221634A13688B431360FFF703FE614BE5
:102CC000614C1878C0B201F0EBF80023A360023326
:102CD000A3605E4B0120236001F0AAF80323A360E8
:102CE00001F03EF8040001F0A3F9050001F038F806
:102CF000574B186001F0F4F9564B1968621A531ECD
:102D0000A14200D213008022D203934201D39B023E
:102D10009B0A3268D16AC90700D478E04E491C0C7E
:102D200009689BB24C4359432402090A64180327DB
:102D30004A49FC3293680A6849489B1A494A4A4EF4
:102D400012684A499B18414A34609A183B400193E3
:102D5000036892089C46019B0A6063440360042B4D
:102D600003D901323B400A6003600B684049E41814
:102D7000200001F055FA3F4F3D493B68C3183B60C6
:102D80002000019301F09CF83B4C2068081838495A
:102D90002060884205D9019B01333B6001F090F827
:102DA000216001F02DF9354B1B78002B0ED001F07E
:102DB0003FF93168324B4A1B1B6812189A4233D2D2
:102DC000591A4919091A2F4801F02AF82E4C237A6A
:102DD000002B0FD001F02CF93168E3684A1B121860
:102DE000934224D9591A4919091A284801F018F8A8
:102DF00000232372264B83F3088800F0A1FF0220F2
:102E000001F0E6F9002001F01BFA01F051F9DC01B4
:102E100099000234641A5900641A09214B43803323
:102E2000CB40A408E41882E7FA218900CBE71949CE
:102E3000DBE7C0466466FF1F0C0AFF1FB641210393
:102E400010000040490AFF1F14100040C409000090
:102E5000100AFF1F340AFF1F380AFF1F200AFF1F36
:102E6000280AFF1F1C0AFF1F4866FF1F240AFF1FB6
:102E7000710200006008FF1F2C0AFF1F1C09FF1FC2
:102E8000E408FF1F00100040740BFF1F3C100040BF
:102E900000000020DC050000A022054B92009B589A
:102EA00010B5002B01D0984710BD00F0A1FFFBE743
:102EB0000000FF1FA122054B92009B5810B5002B6C
:102EC00001D0984710BD00F093FFFBE70000FF1F03
:102ED000A222054B92009B5810B5002B01D09847B9
:102EE00010BD00F085FFFBE70000FF1FA322054B8C
:102EF00092009B5810B5002B01D0984710BD00F0F0
:102F000077FFFBE70000FF1FA422054B92009B58B0
:102F100010B5002B01D0984710BD00F069FFFBE70A
:102F20000000FF1F70B501F083F8514B18600420BA
:102F300001F04EF900F054FF0400C30702D401F081
:102F40002FF870BD00224B4B1A604B4B187801389C
:102F500004282CD800F0C6FE03231B1F27002000E6
:102F600000F0FEFF0128ECD0444C2378042B71D1F3
:102F700001F096F8002806D000F0D2FF582000F0AB
:102F800007FF02232370032001F022F9D9E7200074
:102F900000F03EFFE6E7200000F0D2FFE2E720006D
:102FA00001F04EF8DEE7200000F04AFFDAE701F01A
:102FB0001FF90500012808D1314B1B78053B012B77
:102FC00003D82000FFF768FFCEE72C4B1B78022BBD
:102FD00001D0052B20D1022D28D12A4B9B7BAB435E
:102FE0001CD12000FFF766FF254B18780128BBD1C4
:102FF0006405B9D4234925224B7B034205D1233AEA
:1030000013405A42534126331A000B7D9342ABD9E9
:10301000322001F08DF8A7E7022D07D1184B1B785D
:10302000052B11D12000FFF753FFDDE7012D0BD158
:10303000012B03D12000FFF759FF95E7062B03D1A1
:103040002000FFF761FF8FE7200000F0D1FE022D86
:103050008AD1C9E7032B04D10B4B987C01F000F80F
:1030600091E7072B8FD1094B987B01F079F88AE71C
:103070009C09FF1F9809FF1F9009FF1F2309FF1FCD
:103080001C09FF1FA60BFF1FBC0BFF1FD40BFF1F4C
:10309000FA210A4B0A4A49001A640A4A5A500A4A53
:1030A00004395A50094A08319A64094A5A50094A5F
:1030B0005C315A50084ADA667047C0460000FF1F6C
:1030C0007527FF1F7128FF1F2528FF1F7D23FF1F66
:1030D000E526FF1F011EFF1FD51DFF1F10B500F0C5
:1030E000E9FD10BD8023F7B59C46264B264F019382
:1030F0002649274A274D284C284B02281AD16046DA
:1031000038600868264E3040802636033043086019
:1031100001990978002909D11660224A2A60224AB9
:103120002260E02219689143A03A1BE08021C90285
:103130001160F2E766463E600F68194E3E408027F8
:10314000FF023E430E600199097800290DD11760F6
:1031500001280ED1154A2A60154A2260E02219681A
:103160009143C03A0A431A60F7BD80218902116079
:10317000EEE7E0210F4A02432A600F4A22601A68F4
:103180008A43F0E74B0AFF1FE0000340D8000340EA
:103190009000034000000340500003404000034003
:1031A000FFFFE3FF0280063D804508220180063DC7
:1031B000806608220080069880550822F8B51E4BCC
:1031C00080261A68002014003440324232D11A6836
:1031D0001A4F32431A6001223B68063093433B602A
:1031E00000F026FE0122164D2B681E432E603B6820
:1031F0000A2613433B608027BF00124B1B683B42EB
:1032000011D1013EF6B2FF2E09D17E220E4B1C6871
:103210002B68E40B1440934323432B6005E0082004
:1032200000F006FEE9E7002EEFD180222B6860084F
:1032300093432B60F8BDC046C4F000405CF00040F2
:1032400018F0004068F0004060F0004010B500F059
:10325000A7FF01215820034A00F08AFDFFF7AEFFC7
:1032600010BDC046600AFF1F10B578220021034838
:1032700000F06EFF00F04CFF002010BD6C69FF1FD6
:1032800070B5040000F054FD00230C200B4A01002F
:1032900059438D18515C00290DD0A14208D101235A
:1032A00000246B7000F07CFD00F0AAFF200070BDD0
:1032B00001330A2BEBD11224F6E7C0466C69FF1FDD
:1032C00070B5040000F034FD002319001D000D4A04
:1032D0001078002806D0A0420CD1557001310C3274
:1032E0000A29F5D1002B0AD100F012FF00F088FF67
:1032F000002070BD5078461EB0411B18EEE700F06C
:103300004FFDF3E76C69FF1FF7B504000C200023A5
:1033100084460E4D019267465F43E85D7E19A042E8
:1033200012D000280BD10A4B9C4662461B7808330A
:103330001370019B70707C557160B360FEBD0133EA
:103340000A2BE8D10320F9E70720F7E76C69FF1F94
:103350006869FF1F8021F8B5464BC9051B68C12469
:103360008B60454BFF261A68012313434B61434B87
:10337000A4001A68424B40201A60424B1A68424B24
:103380001A60424B1A59B2431A51C52292009D58F5
:10339000B5432843802598509F583D48ED0107408C
:1033A0003D439D509D5880272D022D0A2943995059
:1033B00080211A59090202400A431A5104341A5949
:1033C000344D3F042A403A4380271A511A593F0688
:1033D0001202120A3A431A5108341A5902400A4397
:1033E0001A51C32292009D58B5432C0080252C43CE
:1033F0009C509D582C0004400C439C509D58254CDB
:1034000025408024240425439D509C588025240277
:10341000240A3C439C50C424A4001A59B2432A43B2
:103420001A511A591202120A17431F5108341A5915
:10343000B24315431D5100251A5902400A431A513F
:1034400004341A59024011431951134C134B1B7881
:10345000DB08AB4201DC0020F8BD2378002B06D04E
:10346000A368002B00D0984701350C34EEE71220FA
:10347000F2E7C0465045FF1F4C45FF1FB0F000402B
:103480006469FF1FB4F000406069FF1F00E100E0C5
:10349000FF00FFFFFFFF00FF6C69FF1F6869FF1F50
:1034A000030010B51F2809D8072200201340072465
:1034B00004490A78A24313430B7010BD0023062071
:1034C000F5E7C0466869FF1F034A044913680020F6
:1034D0000B4013607047C0461CF00040FFFFC1FF67
:1034E000054B06491B780A6805485B0702401B0B21
:1034F000134300200B6070476869FF1F1CF00040F9
:10350000FFFFC1FF70B50C25FFF7EAFF0A4B1C78DF
:103510000A4BE4086543ED18002C01D1200070BD72
:103520002B78002B06D06B68002B00D09847013C0D
:103530000C3DF1E71220F2E76869FF1F6069FF1F89
:1035400007B50422074801A900F034F9019B0133B3
:1035500005D18023044ADB0411680B43136000206B
:103560000EBDC0461C18001114F00040F0B5050057
:103570002026184B87B00493049B002B03D1112401
:10358000200007B0F0BD002102220B000191009144
:10359000052000F0EDFC02230F490A681A42FCD115
:1035A0000596059C631E0593002CFAD10B4A1368FF
:1035B000002BFCDA0F276F440121380000F090FC4B
:1035C0003B782B42DCD0052000F032FC049B013B11
:1035D0000493D1E7FFFFFF0790C8004000C80040F8
:1035E00007B500F0A5FB80220821D205936A01915E
:1035F000002B01D10739916202210C4A1160019917
:10360000481E01900029FAD1033111600531019162
:103610000199481E01900029FAD11160002B02D1B6
:103620008022D205936200F0EBFD07BD00C0004090
:10363000F0B52D4C89B02378002B4FD1FEF762F9FD
:1036400002232A4F03903A681A42FCD120230693A2
:10365000069B5A1E0692002BFAD1254E3368002B8A
:10366000FCDA0120FFF782FF011E02D0112009B011
:10367000F0BD030003220190009005AD9F2000F0F3
:1036800077FC0321280000F02BFC02233A681A4241
:10369000FCD120230793079B5A1E0792002BFAD1D7
:1036A0003368002BFCDA0120FFF760FF0028DDD132
:1036B0000398FEF73BF9AA786B7811041B020B43C1
:1036C00029780B4363601300113B0A49052B07D887
:1036D00001239340A3600B60012323700020C6E701
:1036E00080231B03F6E7C0463845FF1F90C8004003
:1036F00000C800409808FF1F1E4B30B55A68187864
:103700001D4B85B0D31859424B4101210093002332
:1037100000F036FC194B1A4A02259A6300221A65FA
:1037200010325A658022C4219D65164B1648D2027C
:10373000DA6789004258154B80241A4080231B0405
:1037400013434350642341200393E40500F078F9C8
:10375000402000F075F96562039D6B1E0393002DF8
:10376000FAD103236362FFF73BFFA562FFF760FF17
:1037700005B030BD4445FF1F95FFFEF700C800406F
:10378000050001FF04E100E000E100E0FFFF00FFB1
:1037900010B5064B18705960FFF7AEFF00211320DB
:1037A000034AFFF7B1FD002010BDC0464445FF1F8E
:1037B000F936FF1FF0B5040085B003920291FEF7C1
:1037C000A1F8882263035B0B52051A438023DB05B3
:1037D0009D6A8023274F0092BA68002601901B0340
:1037E0009A420CD9F82326001B041E401C4206D026
:1037F0008022214B52025E6219680A431A60002D32
:103800000BD100F095FA02221C4B1A608023DB05D5
:103810005A62013A9A6200F0F3FC0023039A934241
:1038200020D1002D0AD100F083FA144B03221D6031
:103830008023DB055A629D6200F0E2FC8023BA68B7
:103840001B039A4208D9002E06D000220A4B0C49CD
:103850005A621A680A401A600198FEF767F8002059
:1038600005B0F0BD009A0299D2181278CA540133FB
:10387000D4E7C0463845FF1F00C8004000C00040E4
:10388000FFFFFEFFF0B587B0029103920400FEF740
:1038900039F8019000F04CFA802302250122234ED2
:1038A000DB0535605D629A6200F0AAFC204F3B6840
:1038B0002B42FCD120230493049B5A1E0492002B1C
:1038C000FAD11C4D2B68002BFCDA0120FFF74EFECD
:1038D000002802D0112007B0F0BD2000039A029901
:1038E00000F07EFC022304003A681A42FCD1202337
:1038F0000593059B5A1E0592002BFAD12B68002BCD
:10390000FCDA0120FFF732FE051EE3D100F010FAC9
:1039100080230322DB0535605A629D6200F070FC53
:103920000198FEF703F8E0B2D5E7C04600C00040BA
:1039300090C8004000C80040F0B5802687B0040061
:10394000FDF7E0FFF605B36A02250393029000F04D
:10395000EFF90123244F3D607562B36200F050FC23
:10396000224E33682B42FCD120230493049B5A1E21
:103970000492002BFAD11E4D2B68002BFCDA01209B
:10398000FFF7F4FD002802D0112007B0F0BD2000A1
:1039900000F0B6FA0223019032681A42FCD12023CB
:1039A0000593059B5A1E0592002BFAD12B68002B1C
:1039B000FCDA0320FFF7DAFD041EE5D100F0B8F9C8
:1039C00080230322DB053C605A629C6200F018FCF5
:1039D000039B002B01D1FFF703FE0298FDF7A6FF22
:1039E0006B461879D1E7C04600C0004090C800403F
:1039F00000C8004007B5000201910422000A01A995
:103A0000FFF740FF0EBD000073B5050005240B4A0B
:103A1000A3005B429B1819686B46DE1D300000F066
:103A200067FA022804D133782B55013CEFD276BDDA
:103A3000052CFCD00128FAD10230F8E71409001156
:103A40001F2807D8012380228340D20591680B43A9
:103A5000936070473F2808D8012380222038834094
:103A6000D20551690B435361F3E75F28F1D8012375
:103A7000802240388340D205116A0B431362E8E785
:103A80001F2807D8012280218240C9058B689343F3
:103A90008B6070473F2808D801228021203882405F
:103AA000C9054B6993434B61F3E75F28F1D80122C5
:103AB000802140388240C9050B6A93430B62E8E7D6
:103AC0001F2810D880230200DB05153A1968012A47
:103AD00006D820229143196019680A431A6070477A
:103AE00001228240F6E73F2811D880230200DB053F
:103AF000353AD968032A06D810229143D960D9688B
:103B00000A43DA60EBE7012220388240F5E75F28BC
:103B1000E5D842238022181A413B8340D205516ADE
:103B200099435162516A0B435362D8E710B50400C0
:103B3000012813D1A022184992050B685B015B098B
:103B400013430B60154B164A19681140154A0A4376
:103B50001A60402219680A431A6010BD0028FCD17F
:103B600001000A2000F014FA21000B2000F010FAE6
:103B7000C0220A4B920019680A4340211A601A6851
:103B80008A431A60B022044912060B685B015B0984
:103B900013430B60E1E7C04614F000401CF0004006
:103BA0007F00FEFF80FD010072B6074A13680133F3
:103BB00013600422054B1A600023054A136080221B
:103BC000D2055360FEE7C0467808FF1FC0F00040F2
:103BD000C4F00040044B054A1A60054B1A600022ED
:103BE000044B1A607047C046140AFF1F841E000071
:103BF000380AFF1FC4F000400023034A1360034A41
:103C00001360034A1360704754F0004040F10040D5
:103C100044F10040002310B5184C8AB00093019382
:103C20002378012B27D06946012000F079FA00287B
:103C300017D1009B12490293019B06AA0393114BD3
:103C400002A81B680493104B1B68059300F0B8F999
:103C500010220E4906A800F0B3FA002804D1FF2371
:103C6000237000200AB010BD0123094A074902A8A9
:103C7000237000F0A5F90120F4E7C0466866FF1F35
:103C800010290011082900110C2900112029001108
:103C90006C66FF1F13B501246946012000F040FA4D
:103CA000034B00940193FFF7B5FF200016BDC046FB
:103CB000BB0B000010B5FFF79FFFFFF7EBFF0028DD
:103CC00002D0024B984710BDFEE7C046E1A20000BB
:103CD00002B4714649084900095649008E4402BCA5
:103CE0007047C04602B4714649084900095C490062
:103CF0008E4402BC7047C04603B471464908400078
:103D00004900095A49008E4403BC70470000000076
:103D100001B40248844601BC604700BF53B90000AB
:103D200001B40248844601BC604700BFCD0C0100CD
:103D300001B40248844601BC604700BF75A9000079
:103D400001B40248844601BC604700BF7997000077
:103D500001B40248844601BC604700BF0D52010017
:103D600001B40248844601BC604700BF156B0100E6
:103D700001B40248844601BC604700BF01670100EE
:103D800001B40248844601BC604700BFE51201004F
:103D900001B40248844601BC604700BF79120100AB
:103DA00001B40248844601BC604700BF21A900005D
:103DB00001B40248844601BC604700BF5976010047
:103DC00001B40248844601BC604700BF116E000088
:103DD00001B40248844601BC604700BF71B00000D6
:103DE00001B40248844601BC604700BFBD0B01001E
:103DF00001B40248844601BC604700BFE9170100D6
:103E000001B40248844601BC604700BFF9A6000027
:103E100001B40248844601BC604700BF0934010078
:103E200001B40248844601BC604700BF2D6C01000C
:103E300001B40248844601BC604700BF018900000C
:103E400001B40248844601BC604700BFF935010057
:103E500001B40248844601BC604700BFE94C010040
:103E600001B40248844601BC604700BFE9D40000A9
:103E700001B40248844601BC604700BFD5B60011BA
:103E800001B40248844601BC604700BF19FA000033
:103E900001B40248844601BC604700BFD9B00000AD
:103EA00001B40248844601BC604700BF8914010088
:103EB00001B40248844601BC604700BF8B52010038
:103EC00001B40248844601BC604700BF090E0000EF
:103ED00001B40248844601BC604700BF8D11010057
:103EE00001B40248844601BC604700BF3D71010037
:103EF00001B40248844601BC604700BF8D38001100
:103F000001B40248844601BC604700BFA96F0100AC
:103F100001B40248844601BC604700BFE9270000A5
:103F200001B40248844601BC604700BF6DF6000042
:103F300001B40248844601BC604700BF2144000030
:103F400001B40248844601BC604700BF053401004B
:103F500001B40248844601BC604700BF89440000A8
:103F600001B40248844601BC604700BF013401002F
:103F700001B40248844601BC604700BF496D01009E
:103F800001B40248844601BC604700BFC56D010012
:103F900001B40248844601BC604700BFC5A20011BD
:103FA00001B40248844601BC604700BFDD0A01003D
:103FB00001B40248844601BC604700BFF9ED00002F
:103FC00001B40248844601BC604700BFDD3F0000E9
:103FD00001B40248844601BC604700BFC9A9000083
:103FE00001B40248844601BC604700BF8D820000D6
:103FF00001B40248844601BC604700BFBD5C0100BB
:1040000001B40248844601BC604700BFD5440100AA
:1040100001B40248844601BC604700BFE9F60000D5
:1040200001B40248844601BC604700BFE90B0100AF
:1040300001B40248844601BC604700BFC95C01006E
:1040400001B40248844601BC604700BFF535010059
:1040500001B40248844601BC604700BF75F8000007
:1040600001B40248844601BC604700BF4DF900001E
:1040700001B40248844601BC604700BFA9D80000D3
:1040800001B40248844601BC604700BFEDA50000B2
:1040900001B40248844601BC604700BF85C10000EE
:1040A00001B40248844601BC604700BF01D700004C
:1040B00001B40248844601BC604700BF855201003C
:1040C00001B40248844601BC604700BF851201006C
:1040D00001B40248844601BC604700BF9D6A0000ED
:1040E00001B40248844601BC604700BFC1660100BC
:1040F00001B40248844601BC604700BF8937010013
:1041000001B40248844601BC604700BFC1A500005D
:1041100001B40248844601BC604700BFADAE000058
:1041200001B40248844601BC604700BFE1AC000016
:1041300001B40248844601BC604700BF61370100FA
:1041400001B40248844601BC604700BFED6B01002A
:1041500001B40248844601BC604700BFB70E0000AE
:1041600001B40248844601BC604700BFC1F70000AB
:1041700001B40248844601BC604700BF6D0B0100DA
:1041800001B40248844601BC604700BF69110100C8
:1041900001B40248844601BC604700BFC11501005C
:1041A00001B40248844601BC604700BFED680100CD
:1041B00001B40248844601BC604700BF51B800000A
:1041C00001B40248844601BC604700BFCD4C0100E9
:1041D00001B40248844601BC604700BF19070100D2
:1041E00001B40248844601BC604700BF95730100DA
:1041F00001B40248844601BC604700BFDD0C0100E9
:1042000001B40248844601BC604700BF9DA900007C
:1042100001B40248844601BC604700BFA1AF000062
:1042200001B40248844601BC604700BF090E00008B
:1042300001B40248844601BC604700BFB35201008C
:1042400001B40248844601BC604700BF016C010014
:1042500001B40248844601BC604700BFF90D01006B
:104260000200000036C0001101000000E8BD00118E
:104270000200000032C0001101000000A042FF1F38
:1042800002000000F0BD001101000000A863FF1F44
:104290000200000030C00011030000001C63FF1F7B
:1042A000120000000200000036C0001101000000F2
:1042B00030BE00110200000032C0001101000000F9
:1042C0002DBE0011020000003ABE001103000000E4
:1042D0005763FF1F0200000030C000110300000000
:1042E0006C63FF1F0200000032C0001101000000DB
:1042F0002CBE00110200000038BE001103000000B7
:104300002D63FF1F0200000030C0001103000000F9
:104310004E63FF1F0200000036C0001101000000C4
:1043200070BE00110200000032C000110100000048
:10433000E943FF1F0200000082BE001101000000DF
:104340006BBE00110200000032C00011010000002D
:10435000E843FF1F0200000080BE001101000000C2
:104360007463FF1F0200000032C000110100000052
:10437000E743FF1F020000007EBE001101000000A5
:104380005BBE00110200000032C0001101000000FD
:10439000E643FF1F020000007CBE00110100000088
:1043A00056BE00110200000032C0001101000000E2
:1043B000E543FF1F020000007ABE0011010000006B
:1043C00051BE00110200000032C0001101000000C7
:1043D000E443FF1F0200000078BE0011010000004E
:1043E0004CBE00110202020202020000114C001138
:1043F000D74B0011C4BE0011900118001800FFFF38
:104400000701020304050602010600000000000087
:10441000000000000000000000000000000000009C
:1044200000000000000003000200000036C0001180
:104430000100000044BF00110200000032C0001162
:10444000010000009844FF1F020000004EBF001151
:1044500001000000A263FF1F0200000030C0001135
:10446000030000001066FF1F0200000032C00011B0
:10447000010000009844FF1F020000004CBF001123
:1044800001000000A463FF1F0200000030C0001103
:10449000030000000866FF1F12A6A6A60000000089
:1044A0000001000000000111FFFF000050485936D4
:1044B000000000000000000001000000D5BE001157
:1044C0000B000500F7000000B400002800280028B9
:1044D0003075A000A000A000A00000080008E001C6
:1044E000F00010001000100010001000100050002C
:1044F0005000500010001000D00700000000000025
:104500000F0001000500307507001000010081FF59
:1045100000000000FF0000009D740011A572001152
:1045200035700011FFFF0100FF000000B99E00116F
:10453000359C00114D9B00110000000000000000A0
:1045400000000800040000003B0001085902E001DF
:1045500088212800FF0000000200000036C0001182
:1045600001000000FCC000110200000032C0001178
:1045700001000000D545FF1F020000002EC0001101
:1045800001000000246AFF1F0200000032C0001179
:1045900001000000D445FF1F020000002CC00011E4
:1045A00001000000D245FF1F0200000032C00011D0
:1045B00001000000D045FF1F020000002AC00011CA
:1045C00001000000C845FF1F1800180000009001FE
:1045D00002000003020200000200000036C00011C9
:1045E0000100000010C100110200000032C00011E3
:1045F000010000001846FF1F0200000028C0001143
:1046000000000000000000000200000030C00011A7
:0A46100003000000446AFF1F20FFB2
:040000051FFF184180
:00000001FF
